:020000040800F2
:10000000703800200501000865360008CB2E000876
:10001000593100085D100008054300080000000089
:10002000000000000000000000000000153B000878
:10003000CD100008000000006D370008013C0008EA
:100040001F0100081F0100081F0100081F01000810
:100050001F0100081F0100081F0100081F01000800
:100060001F0100081F0100081F0100081F010008F0
:10007000611000087110000881100008911000083C
:100080001F0100081F0100081F0100081F010008D0
:100090001F0100081F0100081F0100081F010008C0
:1000A0001F0100081F0100081F0100081F010008B0
:1000B0001F0100081F0100081F0100081F010008A0
:1000C0001F0100081F0100081F0100081F01000890
:1000D0001F010008854200081F010008C5420008F2
:1000E0001F0100081F0100081F010008DFF810D0E1
:1000F00000F062FC00480047415B0008AFF300805D
:10010000703800200648804706480047FEE7FEE7B3
:10011000FEE7FEE7FEE7FEE7FEE7FEE7FEE7FEE7B7
:100120009F3C0008ED000008202A04DB203A21FA59
:1001300002F00021704721FA02F3D040C2F1200200
:10014000914008431946704740EA01039B0703D0DA
:1001500009E008C9121F08C0042AFAD203E011F806
:10016000013B00F8013B521EF9D27047D2B201E0C8
:1001700000F8012B491EFBD270470022F6E710B5AC
:1001800013460A4604461946FFF7F0FF204610BD05
:10019000421C10F8011B0029FBD1801A704730B5B2
:1001A00004460020034600E05B1C934203D2E05C5F
:1001B000CD5C401BF8D030BD30B50546002003466D
:1001C00000E05B1C934205D2EC5CC85C201A01D1B4
:1001D000002CF6D130BD00000FB400B58DB010A9D1
:1001E00009900B9000914FF0FF300A9000200C9086
:1001F00005480690054807906A4609A80F9900F03F
:10020000A3FA0DB05DF814FB65070008830700082A
:100210002DE9FF5F1D464FF0FF3BD5E901469146B2
:100220005F464FF00008A9697F1C01988847296A3A
:10023000824688470028F6D1BAF1FF3F0CD024F45B
:10024000C064002E19DD600614D5BAF12B0F09D059
:10025000BAF12D0F0ED103E0584604B0BDE8F09F6F
:1002600044F48064A9697F1C01988847761E824601
:10027000002E02DDBAF1300F03D0B9F1000F26D005
:1002800032E0A969761E44F400747F1C0198884707
:100290008246002E05DDBAF1780F06D0BAF1580F6C
:1002A00003D0B9F1000F10D01EE0B9F1000F02D059
:1002B000B9F1100F18D1A969761E24F400747F1CBF
:1002C000019888478246102002E0082000E00A20BA
:1002D000814609E008FB0908A969761E44F4007408
:1002E0007F1C019888478246002E05DD494650460E
:1002F00000F015FA0028EDDAE96901988847A005B1
:1003000002D46FF00100A8E7E00725D1600613D5FD
:10031000600502D5C8F1000000E0404629680A1DCA
:100320002A600968220501D5087015E0220701D569
:10033000088011E008600FE02868011D296000684E
:10034000210502D580F8008006E0210702D5A0F83B
:10035000008001E0C0F8008038467EE72DE9FF4FBD
:10036000087883B09946FF2805D0491C2D2804D071
:100370000024002008E000200BE00124F9E700EB56
:10038000800003EB4000491C0B78FF2BF7D104B130
:10039000404200230293147819461D462D2C01D0AB
:1003A0002B2C04D1521C2D2C13D000240294AA46CD
:1003B0001478FF2C0FD00A25A3FB057801FB0581DB
:1003C0004FF0000C03FB0C11521CE3194AEB010126
:1003D000EEE70124EAE7814453EA010002D019F56F
:1003E000C87F06DA03980021C0E9001107B0BDE814
:1003F000F08F0025AE4E2F46DFF8B882184600F089
:10040000B2FACDE90001B9F1000002DAC9F1000445
:1004100000E004460023A74A1AEB030B42EB045A00
:1004200012E0E00707D02A4633463846414600F03E
:10043000B9F9074688462A4633461046194600F061
:10044000B1F905460E466410002CEAD1DDE9000141
:10045000B9F1000F5A46534606DA00F015FA3A464B
:10046000434600F011FA05E000F09CF93A46434695
:1004700000F098F9029A0AB181F00041039AC2E9AA
:100480000001B3E72DE9FF4F1F468DB0D7E90146C4
:100490004FF0FF382E2045464FF000090B90B96908
:1004A0006D1C0E988847396A824688470028F6D125
:1004B000BAF1FF3F0AD024F4D064002E11DDBAF166
:1004C0002B0F08D0BAF12D0F0BD102E0404611B02E
:1004D0008DE744F48064B9696D1C0E9888478246A4
:1004E000761E6946600501D52D2000E02B208DF891
:1004F000000001F1010B0DF1200809E0B9696D1C44
:100500000E98884782460F9844F40074761E056062
:10051000002E02DDBAF1300FF0D00B998A453ED1A2
:1005200044F0800406E00F99681CA9F1010944F425
:1005300000740860B9696D1C761E0E988847824663
:100540003028F0D02BE00B998A4505D1200603D442
:1005500044F08004761E18E0504604F0DEF808B33C
:100560000DF11301761E44F400748B4508D2AAF1F4
:1005700030000BF8010B200607D5A9F1010003E0BC
:10058000200602D409F101008146A00502D50F9989
:10059000681C0860B9696D1C0E9888478246002E59
:1005A000D1DC53E0002E51DDBAF1650F02D0BAF173
:1005B000450F4BD1A00549D5B9696D1C24F4407491
:1005C000761E0E9888478246002E0CDD2B2804D01C
:1005D000BAF12D0F07D144F48074B9696D1C0E98DF
:1005E00088478246761EE00501D52D2100E02B21AB
:1005F00008F8011BCDF82C8021E00DF12901761EB1
:1006000044F4007488450CD2AAF1300010F0FF00C9
:1006100088F8000002D10B99884509D908F1010832
:1006200006E0E00501D5244801E042F20F70814662
:10063000B9696D1C0E98884782460F980560002E98
:1006400004DD504604F069F80028D6D1F9690E9807
:100650008847FF208BF8000088F8000000200690F3
:1006600007904B466A4608A906A8FFF777FEA00543
:1006700002D46FF001002AE714F0240F0AD0E0073B
:1006800014D1DDE906123868031D3B600068C0E93B
:1006900000120BE0DDE9060100F071F90146E00708
:1006A00004D13868021D3A600068016028460EE7F0
:1006B000000014400000F03FF1D8FFFF2DE9F05F8B
:1006C0000546002092469B468846064681464024C1
:1006D0001BE02846414647462246FFF725FD534684
:1006E0005A46C01A914110D311461846224600F0CE
:1006F00075F92D1A67EB01084F46224601200021AB
:1007000000F06CF917EB00094E41201EA4F1010422
:10071000DFDC484631462A464346BDE8F09F3A288A
:1007200000D2303820F02002412A01D3A2F1370054
:10073000884201D34FF0FF30704700000268114437
:100740001378016018467047D1600449516104492B
:10075000116200211161114600F054B93D070008F3
:10076000FB090008426842B1016811F8013B23B15E
:10077000521EC0E90012184670470121C160881E50
:10078000704742685AB1C368016843B983688B42B5
:1007900005D0491E521CC0E90012002070474FF0DE
:1007A000FF3070472DE9FE4F81EA030404F0004456
:1007B00021F0004100944FF0000B23F0004350EA79
:1007C00001045ED052EA03045BD0C3F30A54C1F3C0
:1007D0000A552C44A4F2F3340194A0FB0254C1F353
:1007E000130141F48011C3F3130343F4801301FB9D
:1007F000024400FB034E840A970A44EA815447EA04
:100800008357A4FB076802958D0A05FB07854FEA0D
:10081000932C04FB0C542705029D4FEA065847EA27
:100820001637B5EB08056EEB070C870E920E47EAFC
:10083000811742EA8312A7FB0201B6EB0B0164EBBE
:1008400000042B0D43EA0C335E1844EB1C50DA46CF
:100850005146E7FB0201C5F313044FEA0B3343EAA9
:1008600014534FEA0432019C43EA0603A4F10C043A
:100870000294009CCDE900B400F0A2FA03B0BDE8F8
:10088000F08F00200146F9E72DE9F04D81EA0304DD
:1008900004F0004B21F0004514464FF0000A23F00D
:1008A000004150EA050220D054EA01021DD0C5F3F0
:1008B0000A570246C5F31303C1F31300C1F30A56E6
:1008C00040F4801543F48013A7EB0608101BD646AE
:1008D00008F2FD3873EB050002D308F1010801E0CE
:1008E00092185B41B8F1000F03DA00200146BDE821
:1008F000F08D00204FF48011064684460EE0171B51
:1009000073EB050705D3121B63EB050306434CEAA3
:10091000010C49084FEA300092185B4150EA010788
:10092000EDD152EA030012D082EA040083EA050105
:10093000084305D0101BAB4106D20122002306E07C
:1009400000224FF0004302E06FF0010253101AEB57
:1009500006004CEB085110EB0A0041EB0B01BDE81F
:10096000F04D00F01EBA0EB540F233420292002262
:10097000CDE90022134600F023FA03B000BD01F0D8
:10098000004330B421F0004150EA010206D00A0DC4
:10099000A2F56072C1F31301002A02DC30BC002012
:1009A0007047440F44EAC104C100E01830BC00EBBA
:1009B000C25000F0BFB90000064C074D06E0E068E9
:1009C00040F0010394E8070098471034AC42F6D396
:1009D000FFF790FB847B0008A47B0008202A04DB3F
:1009E000203A00FA02F1002070479140C2F1200342
:1009F00020FA03F3194390407047C0B24FF4F0510E
:100A000000F02CBA2DE9F34F8BB04FF0000801F144
:100A10000C000C464FF0010B46460DF1080A019000
:100A20006269012101989047051E2DD0252D2CD0FB
:100A3000216A8847C0B16269012101989047216A03
:100A400088470028F7D1411E62690198904700E06D
:100A5000761CA1690B988847216A88470028F7D13E
:100A6000E1690B988847DBE7A1690B98884707463F
:100A7000A84201D1761CD3E7E1690B9888477F1C17
:100A800002D1B8F1000F6FD047E1002762693D46FF
:100A90003946019890472A2804D1626901210198BA
:100AA00090470125DFF888926269012101989047FB
:100AB000A0F130010A290AD24F45E5DC07EB870196
:100AC00000EB4107303FDFD445F01005ECE7E906C5
:100AD00001D46FF000476C280AD04C2814D0682845
:100AE00015D06A280DD074281CD07A281AD01DE0A1
:100AF00062690121019890476C2802D045F00405F5
:100B000014E045F002050DE045F020050AE06269B9
:100B1000012101989047682802D045F0080505E0BA
:100B200045F400656269012101989047C4E90157C5
:100B300065283DD019DC58287AD00CDC452837D000
:100B400004DC252826D0412831D131E046282FD099
:100B500047282CD12CE05B2877D0612828D0632847
:100B60007CD0642823D15AE0D1E06F2848D008DC3B
:100B700066281DD067281BD0692821D06E2816D181
:100B800027E0702845D0732868D0752847D078288A
:100B90000DD14DE0A1690B988847054625283FF403
:100BA00069AFE1690B9888476D1C3FF46AAFB4E008
:100BB00023466A466FF001000B99FFF763FC9FE044
:100BC00045F040006060A80723464FF0000236D48D
:100BD0003EE0E8077FF447AF2068011D2160006810
:100BE000290501D506701BE7290701D5068017E7FF
:100BF000A90703D5F117C0E9006111E706600FE707
:100C000045F040006060A80723464FF0080216D464
:100C10001EE040F60E0125EA0100606016E045F096
:100C200040006060A80723464FF00A0207D40FE097
:100C300045F040006060A80708D5234610226FF0F9
:100C400001000B99AFF300805AE007E02346102221
:100C50006FF001000B99FFF7DBFA51E04FF000094C
:100C60004F464B46632802D05B2807D041E02079ED
:100C7000C00601D40120A06001273AE06269012189
:100C8000019890475E2805D14FF0010962694946F5
:100C900001989047216939B900210A46534643F823
:100CA0002120491C0829FADBB0B3216969B9C117B1
:100CB00000EBD16253110AEB830122F01F02821A6A
:100CC00001200B68904003430B6062690121019889
:100CD00090475D28E8D1B9F1000F09D000205146B6
:100CE00051F82020D24341F82020401C0828F7DB8F
:100CF00002AB224600976FF001000B99AFF3008022
:100D000000280CDA401C08D1BBF1000F05D04FF0D1
:100D1000FF300DB0BDE8F08FFFE74046F9E7E90787
:100D200001D108F1010806444FF0000B78E60000FD
:100D3000CCCCCC0C0029A8BF7047401C490008BF90
:100D400020F00100704710B4B0FA80FC00FA0CF0FB
:100D500050EA010404BF10BC704749B1CCF1200433
:100D600021FA04F411FA0CF118BF012121430843C0
:100D7000A3EB0C01CB1D4FEA00614FEA102042BFEC
:100D8000002010BC704700EBC35010440029A4BFE2
:100D900010BC7047401C490008BF20F0010010BC87
:100DA000704710B5141E73F1000408DA401C41F1BD
:100DB000000192185B411A4301D120F0010010BDDF
:100DC0002DE9F04D92469B4611B1B1FA81F202E055
:100DD000B0FA80F220329046FFF700FE04460F463C
:100DE00040EA0A0041EA0B0153465A46084313D031
:100DF000114653EA010019D0C8F140025046FFF7EE
:100E000093F905460E46504659464246FFF7E6FD21
:100E1000084305D0012004E020463946BDE8F08DA6
:100E20000020054346EAE0762C4337430A986305E1
:100E3000E40AA0EB08000022FD0A44EA47540A3005
:100E400002D500200146E9E7010510196941DDE9F5
:100E5000084500196941BDE8F04DA2E77F2801D996
:100E6000002208E0064A02EB5002C007127800D1C7
:100E7000120902F00F020120904008407047000064
:100E8000F677000870B58C1810F8015B15F00703B1
:100E900001D110F8013B2A1106D110F8012B03E013
:100EA00010F8016B01F8016B5B1EF9D12B0705D41B
:100EB0000023521E0DD401F8013BFAE710F8013B64
:100EC000CB1A921C03E013F8015B01F8015B521E80
:100ED000F9D5A142D8D3002070BD000010B5144947
:100EE000486880471349C86A8047114908688047A5
:100EF00002F006FC1048816A88471048816A8847DA
:100F00000F49486C80470F49486A80470E49D1F81D
:100F1000CC0080470D49C86880470D490868804764
:100F20000349486880470B490BA003F08DFB10BDB7
:100F3000B4110020D8110020E8100020701100200A
:100F4000441000201C140020301300204C140020FA
:100F5000981000201400002025730A0010B50A2202
:100F6000364801883648008802F07EFB012805D10A
:100F7000324800883249088002F0AFFE32222F4802
:100F800001883048008802F06FFB012805D12B480A
:100F900000882C49088002F0B9FE642227480188A5
:100FA0002948008802F060FB012805D12348008809
:100FB0002549088002F090FEC82220480188234875
:100FC000008802F051FB012805D11C4800881F4908
:100FD000088002F091FE4FF4FA72184801881C480C
:100FE000008802F041FB012805D114480088184907
:100FF000088002F083FE4FF47A7210480188154889
:10100000008802F031FB012805D10C480088114905
:10101000088002F063FE4FF4FA62084801880E4827
:10102000008802F021FB012805D1044800880A4904
:10103000088002F062FE02F033FE10BD2C0000209A
:1010400036000020380000203A0000203C0000203C
:101050003E000020400000204200002000BFFEE7CC
:1010600010B5024800F0DCF910BD00002C1600207D
:1010700010B5024800F0D4F910BD0000E8150020BA
:1010800010B5024800F0CCF910BD0000A4150020F6
:1010900010B5024800F0C4F910BD00006015002032
:1010A00030B590F840500124AC40C56B6C600468CA
:1010B00063604468102C04D10468A2600468E16095
:1010C00003E00468A1600468E26030BD70477047C7
:1010D00010B50446204600F0F3FA10BD38B532488A
:1010E0000068807B401CC0B28DF800002E4800686C
:1010F000C07B401CC0B28DF801002B480068007C0A
:10110000401CC0B28DF8020027480068407C401C9B
:10111000C0B28DF803006A460C21002003F044FAA7
:1011200001220021084603F0FFF9012211460020A8
:1011300003F0FAF9052000F0C3FA0321002002F0C1
:10114000E7FB132806D010220121002003F0ECF960
:10115000002038BD04220121002003F0E5F900BF82
:1011600000240221002002F0D3FB044624B1E2B2A5
:101170000221002003F0D8F9052000F0A1FA04F0C4
:101180000800082801D10020E3E70621002002F032
:10119000BFFBFF2806D010220121002003F0C4F974
:1011A000FF20D6E7DCE700009410002072B600BFF5
:1011B000FEE700000021074AD1610749096941F0B3
:1011C0000401054A11611146096941F040011161AC
:1011D0007047000070160020002002400021074ADE
:1011E000D1610749096941F00201054A11611146BF
:1011F0004861096941F04001116170477016002093
:10120000002002400022054BDA61054A126942F0D3
:101210000102034B1A610180704700007016002024
:101220000020024000201E49C96801F0100139B1B8
:101230001C49C96941F002011A4AD16140F010000D
:101240001749C96801F0040139B11649C96941F06B
:101250000101144AD16140F004001149C96901F04B
:10126000010169B10F49C96941F004010D4AD16119
:1012700000BF0B49C96921F00101094AD16100BFD2
:1012800000BF40F20111884206D10549C96921F029
:101290000101034AD16101E00149C86000BF704704
:1012A000002002407016002070B5044600F096FC45
:1012B000054609E0601C38B124B100F08FFC401BEA
:1012C000A04201D9032070BD1248C06800F001009F
:1012D0000028EFD10F48C06800F0200020B100BF07
:1012E00020200C49C86000BF0A48C06800F0100008
:1012F00048B90848C06900F0010020B90548C06835
:1013000000F0040018B1FFF78DFF0120DBE700209B
:10131000D9E70000002002400146002291F8210098
:10132000022808D00420886300BF002081F8200034
:1013300000BF012070470868006820F00E000B68AD
:1013400018600868006820F001000B68186091F8C8
:10135000403001209840CB6B5860012081F821007B
:1013600000BF002081F8200000BF1046E2E7000027
:1013700070B50446002594F82100022803D004200B
:10138000A063012548E02068006820F00E00216875
:1013900008602068006820F00100216808601F498B
:1013A0002068884201D1012026E01C4914312068C0
:1013B000884201D110201FE0184928312068884256
:1013C00001D1801518E015493C312068884201D1CF
:1013D000801411E0114950312068884202D14FF445
:1013E000803009E00D4964312068884202D14FF411
:1013F000801001E04FF080700849083948600120F2
:1014000084F8210000BF002084F8200000BF606B3A
:1014100010B12046616B8847284670BD0800024025
:1014200070B50446E06B05682068066894F84010C3
:10143000042088402840002846D006F004000028F8
:1014400042D02068006800F0200028B920680068B9
:1014500020F004002168086057492068884201D1C3
:10146000042027E0544914312068884201D14020EB
:1014700020E0514928312068884201D1001519E047
:101480004D493C312068884202D14FF4804011E040
:10149000494950312068884202D14FF4802009E048
:1014A000454964312068884202D14FF4800001E050
:1014B0004FF08060404908394860E06A00287AD0DF
:1014C0002046E16A884776E094F840100220884080
:1014D0002840A0B306F0020088B32068006800F03E
:1014E000200040B92068006820F00A0021680860E8
:1014F000012084F8210030492068884201D102206F
:1015000028E02D4914312068884201D1202021E0B3
:10151000294928312068884201D140151AE026491E
:101520003C312068884202D14FF4005012E0224939
:1015300050312068884203D14FF400300AE017E0B0
:101540001D4964312068884202D14FF4001001E047
:101550004FF0007018490839486000BF002084F837
:10156000200000BFA06A30B32046A16A884722E06D
:1015700094F84010082088402840E0B106F00800A8
:10158000C8B12068006820F00E002168086094F857
:10159000401001208840E16B48600120A06384F87E
:1015A000210000BF002084F8200000BF206B10B194
:1015B0002046216B884770BD08000240014600228A
:1015C00009B901207047164B0868C01A1423B0FBF4
:1015D000F3F08000086412480838C863022081F8DC
:1015E00021000868026843F6F0708243D1E90103E4
:1015F0001843CB6818430B6918434B6918438B6930
:101600001843CB69184302430868026000208863CE
:10161000012081F82100002081F8200000BFD1E7DF
:10162000080002402DE9F04104460D4616461F46CB
:101630004FF0000800BF94F82000012802D10220DA
:10164000BDE8F081012084F8200000BF94F821005B
:1016500001282CD1022084F821000020A0632068FA
:10166000006820F00100216808603B4632462946A8
:101670002046FFF715FDE06A30B12068006840F0B1
:101680000E00216808600BE02068006820F004006C
:10169000216808602068006840F00A00216808603E
:1016A0002068006840F001002168086006E000BF83
:1016B000002084F8200000BF4FF002084046BFE73A
:1016C00070B5044600F08AFA06462546681C10B13B
:1016D00004480078054400BF00F080FA801BA8424F
:1016E000FAD370BD080000202DE9F04104460E46F3
:1016F0000127002500BF2648007E012802D10220D4
:10170000BDE8F08101202249087600BF2068022848
:1017100013D14CF25030FFF7C7FD90BB0120FFF70B
:1017200049FD4CF25030FFF7BFFD074619480069EC
:1017300020F004001749086123E04CF25030FFF715
:10174000B3FDF0B94FF0FF303060A56812E02846D5
:10175000FFF744FD4CF25030FFF7A6FD07460D4859
:10176000006920F002000B4908610FB1356007E005
:1017700005F58065D4E9021001EB8020A842E6D887
:1017800000BF00BF00200249087600BF3846B7E717
:1017900070160020002002400348006940F08000DD
:1017A0000149086100207047002002402DE9FE4FEA
:1017B00005468B46174698460126002400200290D5
:1017C00000BF2448007E012802D10220BDE8FE8F20
:1017D00001202049087600BF4CF25030FFF764FD2D
:1017E000064686BB012D02D10120029006E0022DA3
:1017F00002D10220029001E00420029000241EE0A9
:101800002201B946C24648465146FEF78DFC80B2D9
:101810000190022000FB04B000900199FFF7F2FC58
:101820004CF25030FFF740FD06460B48006920F0AF
:1018300001000949086106B104E0601CC4B20298C5
:101840008442DDDB00BF00BF00200249087600BFF4
:101850003046BBE7701600200020024000200849F7
:10186000096901F0800151B10649054A51600649F4
:1018700051601146096901F0800101B101207047F2
:101880000020024023016745AB89EFCD2DE9F847E1
:101890000346002294466EE14FF0010808FA02F474
:1018A000D1F8008008EA0400A0427DD1DFF8DCA274
:1018B000D1F80480A8EB0A09D0453AD014DCB8F17D
:1018C000030F50D009DCB8F1000F31D0B8F1010F8F
:1018D0001CD0B8F1020F49D120E0B8F1110F18D097
:1018E000B8F1120F42D11EE0B9F5881F25D006DCF1
:1018F000B9F5803F20D0B9F5801F37D11AE0B9F58E
:10190000001F18D0B9F5041F30D117E0D1F80CC072
:101910002DE0D1F80C8008F1040C28E0D1F80C80FF
:1019200008F1080C23E0D1F80C8008F10C0C1EE043
:1019300000BF00BF00BF00BF00BF00BFD1F80880DC
:10194000B8F1000F02D14FF0040C0BE0D1F8088081
:10195000B8F1010F03D14FF0080C1C6102E04FF009
:10196000080C5C6103E04FF0000C00E000BF00BF1A
:10197000FF2801D8984601E003F104084646FF28F5
:1019800002D84FEA820803E0A2F108084FEA88086B
:101990004746D6F800804FF00F0909FA07F928EA00
:1019A00009080CFA07F900E088E048EA0908C6F8D7
:1019B0000080D1F8048008F08058B8F1805F7DD1B4
:1019C00000BFDFF8CC81D8F8188048F00108DFF8B4
:1019D000C091C9F81880C846D8F8188008F00108E6
:1019E000CDF8008000BF00BF4FEAB9384FEA920936
:1019F00058F829504FEA82784FEA18794FF00F08CB
:101A000008FA09F825EA0805DFF88881434502D17C
:101A10004FF0000816E0DFF88081434502D14FF017
:101A200001080FE0DFF87481434502D14FF002084E
:101A300008E0DFF86C81434502D14FF0030801E074
:101A40004FF004084FEA82794FEA197908FA09F849
:101A500048EA0505DFF84C814FEA920948F8295019
:101A6000D1F8048008F48018B8F5801F0AD1DFF897
:101A70003881D8F8008048EA0008DFF82C91C9F8CE
:101A8000008009E0DFF82081D8F8008028EA00080B
:101A9000DFF81491C9F80080D1F8048008F4001828
:101AA000B8F5001F10D1DFF8008108F10408D8F85C
:101AB000008048EA0008DFF8F09000E05AE009F101
:101AC0000409C9F800800DE0DFF8DC8008F10408A3
:101AD000D8F8008028EA0008DFF8CC9009F1040962
:101AE000C9F80080D1F8048008F40038B8F5003F48
:101AF0000ED1DFF8B480A8F10408D8F8008048EAD5
:101B00000008DFF8A490A9F10409C9F800800DE0ED
:101B1000DFF89480A8F10408D8F8008028EA0008CB
:101B2000DFF88490A9F10409C9F80080D1F8048095
:101B300008F48038B8F5803F0ED1DFF86C80A8F14A
:101B40000808D8F8008048EA0008DFF85C90A9F19E
:101B50000809C9F800800DE0DFF84C80A8F10808FA
:101B6000D8F8008028EA0008DFF83C90A9F10809BD
:101B7000C9F80080521CD1F8008028FA02F8B8F1A8
:101B8000000F7FF489AEBDE8F88700000000111057
:101B90000010024000080140000C0140001001400C
:101BA0000014014008000140080401400246936807
:101BB0000B400BB1012000E00020704710B5C26857
:101BC00021EA020302EA010443EA0443036110BD6F
:101BD0000AB1016101E00B0403617047014800682C
:101BE000704700000000002070B504460CB90120C9
:101BF00070BD4CF6CC402168086045F25550216814
:101C00000860D4E9001048602168A0688860FFF788
:101C1000E5FF05460DE0FFF7E1FF401B41F23C31D7
:101C2000884206D92068C06800F0030008B103208C
:101C3000DEE72068C06800F003000028EBD14AF618
:101C4000AA20216808600020D2E701464AF6AA20AF
:101C50000A6810600020704703480068034909784B
:101C60000844014908607047000000200800002077
:101C700010B50848006840F01000064908600320CD
:101C800000F0A8F80F2000F007F800F02BF8002073
:101C900010BD00000020024070B504460E480078D8
:101CA0004FF47A71B1FBF0F00C490968B1FBF0F523
:101CB000284600F07AFD08B1012070BD102C07D233
:101CC00000222146501E00F047F80548046001E05C
:101CD0000120F2E70020F0E7080000200C000020BF
:101CE0000400002008B500BF1148806940F00100E1
:101CF0000F4988610846806900F00100009000BF2C
:101D000000BF00BF0846C06940F08050C861084667
:101D1000C06900F08050009000BF00BF00BF0549BF
:101D2000486820F0E06040F00070486000BF08BDE7
:101D3000001002400000014001460846002809DB6F
:101D400000F01F0301229A4043099B0003F1E023A6
:101D5000C3F8002100BF70472DE9F05F80460D46B3
:101D60001646002702F0AEFC074639462A4633469F
:101D700001F00700C0F1070ABAF1040F02D94FF0D1
:101D8000040A01E0C0F1070AD14600F1040ABAF1E1
:101D9000070F02D24FF0000A01E0A0F1030AD44677
:101DA0004FF0010A0AFA09FAAAF1010A0AEA020A3C
:101DB0000AFA0CFA4FF0010B0BFA0CFBABF1010B1A
:101DC0000BEA030B4AEA0B042146404602F082FC70
:101DD000BDE8F09F00BF00F00702064B19684FF600
:101DE000FF031940044B0B4343EA0221014B1960E6
:101DF00000BF70470CED00E00000FA0570B5044626
:101E00000D460CB9012070BD5A48006800F007006B
:101E1000A8420ED25748006820F0070028435549D1
:101E200008600846006800F00700A84201D00120C1
:101E3000E9E7207800F0020002281DD1207800F0A8
:101E40000400042805D14C48406840F4E0604A4949
:101E50004860207800F00800082805D1464840680E
:101E600040F46050444948604348406820F0F00026
:101E7000A168084340494860207800F0010078B329
:101E80006068012806D13C48006800F4003090B931
:101E90000120B8E76068022806D13748006800F0E2
:101EA000007040B90120AEE73348006800F002003E
:101EB00008B90120A7E73048406820F003006168B6
:101EC00008432D494860FFF789FE064609E0FFF701
:101ED00085FE801B41F28831884202D9032092E7B7
:101EE00007E02548406800F00C006168B0EB810F06
:101EF000EDD12048006800F00700A8420ED91D4827
:101F0000006820F0070028431A4908600846006866
:101F100000F00700A84201D0012074E7207800F00B
:101F20000400042807D11448406820F4E060E16808
:101F3000084311494860207800F00800082808D1BB
:101F40000D48406820F46050216940EAC1000A4908
:101F5000486000F03FF808494968C1F30311074A97
:101F6000515CC8400649086006480068FFF794FEC7
:101F7000002048E70020024000100240DE77000801
:101F80000C00002004000020014800687047000099
:101F90000C00002000B5FFF7F7FF04494968C1F3C2
:101FA0000221034A515CC84000BD000000100240FD
:101FB000EE77000800B5FFF7E7FF04494968C1F371
:101FC000C221034A515CC84000BD0000001002401D
:101FD000EE77000870B500210022002400230020C5
:101FE000134D696801F00C05F5B1042D02D0082DE0
:101FF00019D101E00F4819E00F4DC1F38346AB5DE5
:1020000001F4803555B10A4D6D68C5F340450B4E5E
:10201000725D084D5D43B5FBF2F402E0084D03FB31
:1020200005F4204602E000BF024800BF00BF70BDBB
:102030000010024000127A00CC770008DC7700081C
:1020400000093D00F8B504460CB90120F8BD207820
:1020500000F00100002878D0F848406800F00C003B
:1020600004280CD0F548406800F00C00082811D175
:10207000F248406800F48030B0F5803F0AD1EF4864
:10208000006800F4003000285FD0606800285CD150
:102090000120DBE700BF6068B0F5803F06D1E7486C
:1020A000006840F48030E549086028E0606858B96D
:1020B000E248006820F48030E04908600846006883
:1020C00020F4802008601AE06068B0F5A02F0BD1E2
:1020D000DA48006840F48020D84908600846006863
:1020E00040F4803008600AE0D448006820F4803072
:1020F000D24908600846006820F48020086000BFCC
:10210000606888B1FFF76AFD054606E0FFF766FDE7
:10211000401B642801D9032098E7C848006800F4F0
:1021200000300028F2D010E0FFF758FD054606E029
:10213000FFF754FD401B642801D9032086E7BF4800
:10214000006800F400300028F2D1207800F002008E
:10215000022857D1B948406800F00C0050B1B74888
:10216000406800F00C00082818D1B448406800F41A
:10217000803098B9B148006800F0020020B12069B1
:10218000012801D0012061E7AC48006820F0F80088
:10219000616940EAC100A949086033E02069E8B1FB
:1021A0000120A7490860FFF719FD054606E0FFF783
:1021B00015FD401B022801D9032047E79F4800680E
:1021C00000F002000028F2D09C48006820F0F800DF
:1021D000616940EAC1009949086013E0002098490C
:1021E0000860FFF7FBFC054606E0FFF7F7FC401B25
:1021F000022801D9032029E79048006800F0020076
:102200000028F2D1207800F0080008282DD1A0691C
:10221000B8B101208B490860FFF7E0FC054606E0F5
:10222000FFF7DCFC401B022801D903200EE783489E
:10223000406A00F002000028F2D0012001F098FA74
:1022400013E000207F490860FFF7C8FC054606E060
:10225000FFF7C4FC401B022801D90320F6E67748AB
:10226000406A00F002000028F2D1207800F004005B
:10227000042873D100277148C06900F0805070B9FC
:1022800000BF6E48C06940F080506C49C861084684
:10229000C06900F08050009000BF00BF01276A486D
:1022A000006800F48070B0B96748006840F480703E
:1022B00065490860FFF792FC054606E0FFF78EFCD3
:1022C000401B642801D90320C0E65F48006800F481
:1022D00080700028F2D000BFE068012806D157487E
:1022E000006A40F001005549086227E0E06858B9EB
:1022F0005248006A20F00100504908620846006A0E
:1023000020F00400086219E0E06805280BD14B4872
:10231000006A40F00400494908620846006A40F03B
:10232000010008620AE04548006A20F001004349C4
:1023300008620846006A20F00400086200BFE068F6
:10234000A0B1FFF74BFC054609E0FFF747FC401B37
:1023500041F28831884202D9032077E622E03748EB
:10236000006A00F002000028EFD012E0FFF736FC10
:10237000054608E0FFF732FC401B41F288318842F5
:1023800001D9032062E62D48006A00F0020000280F
:10239000F0D1012F05D12948C06920F0805027498C
:1023A000C86100BFE069C8B32448406800F00C0071
:1023B000082860D0E069022848D10020204908663A
:1023C000FFF70CFC054606E0FFF708FC401B02285F
:1023D00001D903203AE61948006800F0007000288F
:1023E000F2D1206AB0F5803F07D11448406820F44C
:1023F0000030A168084311494860D4E90801084346
:102400000E49496821F4741108430C4948600120C1
:102410000B490866FFF7E2FB054607E03DE0FFF7E2
:10242000DDFB401B022801D903200FE603480068AA
:1024300000F000700028F2D02FE0000000100240F1
:1024400000004242800442420070004000201449D3
:102450000866FFF7C3FB054606E0FFF7BFFB401B1E
:10246000022801D90320F1E50E48006800F0007051
:102470000028F2D111E0E069012800D1E6E5094821
:10248000466806F48031206A814204D106F4701156
:10249000606A814201D00120D8E50020D6E5000025
:1024A000000042420010024010B504460CB9012061
:1024B00010BD606A38B96068B0F5827F00D105E070
:1024C0000021E16102E00021216161610021A1623E
:1024D00094F8510028B9002084F85000204600F0FC
:1024E00043F8022084F851002068006820F0400082
:1024F00021680860A08800F48270218901F40441F9
:102500000843A18901F400610843217C01F0020124
:102510000843217D01F001010843218B01F4007182
:102520000843217F01F0380108432021095D01F0B3
:1025300080010843218D01F400510843216808609F
:102540000421A06901EA1040216848602068C06940
:1025500020F400602168C86100206065012084F8D3
:1025600051000020A4E7000010B586B0044600200A
:1025700002900390049005901949206888422DD15B
:1025800000BF1848806940F48050164988610846A9
:10259000806900F48050019000BF00BF00BF084672
:1025A000806940F0040088610846806900F00400FA
:1025B000019000BF00BFA0200290022003900320E2
:1025C000059002A90848FFF761F940200290002019
:1025D0000390049002A90448FFF758F906B010BD13
:1025E0000030014000100240000801402DE9F8438E
:1025F00004460F4616461D46FFF7F0FA8046B146E0
:1026000094F85100012802D00220BDE8F88307B1F8
:102610000EB90120F9E700BF94F85000012801D15C
:102620000220F2E7012084F8500000BF032084F864
:102630005100002060652763A686E686A063A08718
:10264000E08760642064A068B0F5004F0BD120687B
:10265000006820F04000216808602068006840F4AD
:102660008040216808602068006800F04000402831
:1026700005D02068006840F0400021680860E068EC
:10268000B0F5006F37D1606810B1B9F1010F09D111
:10269000206B00882168C860206B801C2063E08E5E
:1026A000401EE08623E02068806800F002000228D7
:1026B0000AD1206B00882168C860206B801C2063D1
:1026C000E08E401EE08612E0FFF788FAA0EB0800DB
:1026D000A84201D3681C00B94DB9012084F851000B
:1026E00000BF002084F8500000BF03208DE7E08E7B
:1026F0000028D8D136E0606810B1B9F1010F09D1D6
:10270000206B007821680873206B401C2063E08EEA
:10271000401EE08623E02068806800F00200022866
:102720000AD1206B007821680873206B401C20635D
:10273000E08E401EE08612E0FFF750FAA0EB0800A2
:10274000A84201D3681C00B94DB9012084F851009A
:1027500000BF002084F8500000BF032055E7E08E42
:102760000028D8D142462946204601F044F908B154
:1027700020206065A06850B900BF0020009020684C
:10278000C068009020688068009000BF00BF0120F2
:1027900084F8510000BF002084F8500000BF606D35
:1027A00008B1012031E700202FE770B50446254627
:1027B000681EB0F1807F01D301200FE0681E4FF04A
:1027C000E02148610F214FF0FF3001F083FF00202E
:1027D0004FF0E021886107200861002070BD70473C
:1027E00070B50446002520684069C0F3C01594F810
:1027F0004100212817D1B5B100BF00BF21681431B5
:1028000051E8001F21F080002168143141E80002E6
:10281000002AF3D100BFA06B10B1A06BFEF77CFDC6
:10282000204601F08BFB20684069C0F3801594F8C6
:102830004200222817D1B5B100BF00BF2168143172
:1028400051E8001F21F040002168143141E80002E6
:10285000002AF3D100BFE06B10B1E06BFEF75CFD26
:10286000204601F025FB002070BD70472DE9F84F90
:102870000446206805682068C668206847694FF0EC
:102880000009CA4605F00F09B9F1000F0AD105F099
:10289000200038B106F0200020B1204601F061FB95
:1028A000BDE8F88FB9F1000F7BD007F0010018B92F
:1028B00006F49070002874D005F0010030B106F4E1
:1028C000807018B1606C40F00100606405F0040095
:1028D00030B107F0010018B1606C40F00200606494
:1028E00005F0020030B107F0010018B1606C40F053
:1028F0000400606405F0080048B106F0200010B93B
:1029000007F0010018B1606C40F008006064606C72
:10291000002845D005F0200028B106F0200010B1B5
:10292000204601F01EFB20684069C0F3801A606CED
:1029300000F0080010B9BAF1000F2CD0204601F0C9
:10294000B7FA2068406900F0400000B300BF00BF44
:102950002168143151E8001F21F040002168143132
:1029600041E80002002AF3D100BFE06B50B1774884
:10297000E16B4863E06BFEF7FBFC88B1E06B416BF9
:1029800088470DE02046FFF770FF09E009E0204688
:10299000FFF76BFF04E02046FFF767FF002060644D
:1029A0007EE7206B012877D105F01000002873D056
:1029B00006F010000028FAD000BF00200090206828
:1029C0000068009020684068009000BF00BF206849
:1029D000406900F0400000285FD0E06B006840686C
:1029E0001FFA80F8B8F1000F55D0A08D404552DD98
:1029F000A4F82E80E06B8069202843D000BF00BF80
:102A000021680C3151E8001F21F4807021680C31DD
:102A100041E80002002AF3D100BF00BF00BF2168D7
:102A2000143151E8001F21F001002168143141E800
:102A30000002002AF3D100BF00BF00BF216814319B
:102A400051E8001F21F040002168143141E80002E4
:102A5000002AF3D100BF202084F842000020206328
:102A600000BF00BF21680C3151E8001F21F01000A9
:102A700021680C3141E80002002AF3D100BFE06B6D
:102A8000FEF74AFC02206063A08DE28D801A81B2BD
:102A90002046FFF7A4FE03E742E0A08DE18D401A37
:102AA0001FFA80F8E08DD0B3B8F1000F37D000BF27
:102AB00000BF21680C3151E8001F21F4907021689B
:102AC0000C3141E80002002AF3D100BF00BF00BF73
:102AD0002168143151E8001F21F0010021681431F0
:102AE00041E80002002AF3D100BF202084F8420010
:102AF0000020206300BF00BF21680C3151E8001F97
:102B000021F0100021680C3141E80002002AF3D1C5
:102B100000BF0220606341462046FFF760FEBFE62B
:102B200005F0800030B106F0800018B1204601F0B9
:102B300079FBB5E605F0400030B106F0400018B171
:102B4000204601F0EBF9ABE600BFA9E60F3D000817
:102B500010B504460CB9012010BDA06900B100E019
:102B600000BF94F8410028B9002084F840002046B6
:102B700000F02AF8242084F841002068C06820F47E
:102B800000502168C860204601F06AFA2068006998
:102B900020F49040216808612068406920F02A00F4
:102BA000216848612068C06840F400502168C8600E
:102BB00000206064202084F8410084F84200002056
:102BC000606300BFC8E7000010B586B0044600206F
:102BD00002900390049005906F49206888426AD162
:102BE00000BF6E48806940F480406C4988610846A7
:102BF000806900F48040019000BF00BF00BF08461C
:102C0000806940F0040088610846806900F0040093
:102C1000019000BF00BF48150290022003900320DE
:102C2000059002A95E48FEF731FE4FF480600290E5
:102C300000200390049002A95948FEF727FE594846
:102C40005949086000204860002157488160802170
:102C5000C1600021016141618161C161FEF7AEFC8B
:102C600008B1FEF7A3FA00BF4F48E063446200BF1B
:102C70004C4814384D4908601020486000214B48EA
:102C800081608021C1600021016141618161C16178
:102C9000FEF794FC08B1FEF789FA00BF4348A06331
:102CA000446200BF002211462520FFF755F8252079
:102CB000FFF742F86EE03E49206888426AD100BFC3
:102CC0003648C06940F480203449C8610846C0696C
:102CD00000F48020019000BF00BF00BF084680695B
:102CE00040F0080088610846806900F00800019003
:102CF00000BF00BF0815029002200390032005903A
:102D000002A92C48FEF7C2FD4FF40060029000209B
:102D10000390049002A92748FEF7B8FD21482838FF
:102D200025490860002048600021234881608021F7
:102D3000C1600021016141618161C161FEF73EFC1A
:102D400008B1FEF733FA00BF1B48E063446200BFDE
:102D500014483C3819490860102048600021174881
:102D600081608021C1600021016141618161C16197
:102D7000FEF724FC08B1FEF719FA00BF0F48A06364
:102D8000446200BF002211462720FEF7E5FF2720FE
:102D9000FEF7D2FF06B010BD00380140001002401F
:102DA000000801405800024060150020A4150020D2
:102DB00000480040000C0140E81500202C160020BF
:102DC00070B504460D46164694F8420020280BD1F3
:102DD00005B10EB9012070BD00202063324629469E
:102DE000204601F0BBF9F6E70220F4E77047704790
:102DF000F7B50446154694F84100202836D10198CD
:102E000000B10DB90120FEBD01982062A584E584C2
:102E100000206064212084F841001548A16B88627D
:102E20001448A16BC8621448A16B08630020A16B11
:102E3000486301AE23681A1D31682B46A06BFEF76C
:102E4000F1FB6FF040002168086000BF00BF2168FF
:102E5000143151E8001F41F080002168143141E82D
:102E60000002002AF3D100BF0020CCE70220CAE70D
:102E70004B3E0008A33E0008233D000810B5044661
:102E80000B492068884203D10A48016B88470EE04D
:102E900009492068884203D10848016B884706E049
:102EA00007492068884202D10648016B884710BD57
:102EB00000380140E8100020004400402C110020A0
:102EC0000048004070110020704700BFFEE7014637
:102ED0000A2291FBF2F302FB13120A2391FBF3F394
:102EE00002EB0312D0B2704708B500BF1648406924
:102EF00040F00100144948610846406900F00100B3
:102F0000009000BF00BF002211460C20FEF724FFF6
:102F10000C20FEF711FF002211460D20FEF71CFFCA
:102F20000D20FEF709FF002211460E20FEF714FFC8
:102F30000E20FEF701FF002211460F20FEF70CFFC6
:102F40000F20FEF7F9FE08BD0010024000B585B065
:102F50000020019002900390049000BF43488069D4
:102F600040F01000414988610846806900F0100077
:102F7000009000BF00BF00BF0846806940F02000FD
:102F800088610846806900F02000009000BF00BF03
:102F900000BF0846806940F00400886108468069E7
:102FA00000F00400009000BF00BF00BF0846806929
:102FB00040F0080088610846806900F00800009031
:102FC00000BF00BF00224FF400512948FEF700FE69
:102FD000002248F218012748FEF7FAFD01221146A7
:102FE0002548FEF7F5FD0022E0212348FEF7F0FD1D
:102FF0004FF4005001900120029000200390022025
:10300000049001A91A48FEF741FC18200190012004
:103010000290002003900220049001A91548FEF7B9
:1030200035FC0120019002900220039003200490BF
:1030300001A91148FEF72AFC4FF40040019001203D
:10304000029002200390049001A90A48FEF71EFC9A
:10305000E0200190012002900020039002200490C3
:1030600001A90548FEF712FC05B000BD00100240A2
:103070000010014000080140000C014010B5074855
:1030800007490860062048604FF4EA7104488160EF
:10309000FEF7AAFD08B1FEF789F810BD0030004028
:1030A0006C14002010B50E480E4908604FF4827071
:1030B000486000210B488160C160016141614FF4AB
:1030C000007181610821C161002101624162816258
:1030D0000A21C162FFF7E8F908B1FEF767F810BDF1
:1030E000003001407814002010B50B480B490860EF
:1030F0004FF416504860002108488160C1600161AA
:103100000C21416100218161C161FFF721FD08B1FE
:10311000FEF74CF810BD000000380140D01400202C
:1031200010B50B480B4908604FF416504860002159
:1031300008488160C16001610C2141610021816109
:10314000C161FFF705FD08B1FEF730F810BD0000C2
:10315000004800401815002000BFFEE72DE9F041AF
:1031600004460D46164614B90020BDE8F081082E2D
:1031700001DA0020F9E7B01E81B2284600F054FAC7
:103180000746A81910F8018C4FF6FF7000EA0828CE
:10319000A81910F8020C40EA0808B84501D0002030
:1031A000E3E72878207068786070A8780002608073
:1031B0006088E978084360806078062802D1281D7D
:1031C000A06013E06078102809D128790002A0805F
:1031D000A08869790843A080E81DA06006E02879EE
:1031E0000002A080A08869790843A0800120BCE784
:1031F00010B501461B2949D2DFE801F00E0F10116E
:10320000121314151617181921222324252B2C2DDF
:103210002E333C3D3E3F450000BF00BF00BF00BF16
:1032200000BF00BF00BF00BF00BF00BF00BF194B01
:1032300003EB41025378147843EA042028E000BFEE
:1032400000BF00BF00BFA1F10C03134C34F8130002
:103250001EE000BF00BF00BFA1F111030F4CE05CF6
:1032600016E00E4B0E3B93F8284093F8273044EAC3
:1032700003200DE000BF00BF00BFA1F11604074B03
:103280000B33185D04E0064B188C01E0002000BFF2
:1032900000BF10BD14000020EE11002052000020DD
:1032A0001C1400202DE9F04781468A4652464946C3
:1032B000A548FFF753FF08B9BDE8F087A3480068A9
:1032C0000078A1490978884200D0F5E74FF000085E
:1032D0009D48407806287CD004DC032807D00428C9
:1032E00078D105E0102876D04128F9D13BE000BF25
:1032F0009548478800789649087093484078487008
:10330000914800794006000E887000250FE038468D
:10331000FFF76EFF0646310A6800C01C8C4A115444
:103320006800001D1654781C87B2681CC5B2864818
:103330008088A842EBDC86488078C11C844800F075
:1033400073F9044682488078C01C814A1454210ACB
:1033500010468078001D115410468078401D11469B
:10336000A1F80002CBE078484788007878490870D7
:1033700075484078487074484088001288707248D8
:103380008078C87070488088C0F3D71008716E4884
:1033900000794006000E487100250FE03846FFF71F
:1033A00027FF0646310A6800801D694A11546800EB
:1033B000C01D1654781C87B2681CC5B2624880884C
:1033C000A842EBDC604880884000801D81B26048E4
:1033D00002E018E08EE04BE000F026F904465A487F
:1033E00080884000801D5A4A1454210A564880881B
:1033F0004000C01D115454488088400008301146D8
:10340000A1F800027BE050484788806840784E4928
:103410008968097840EA01263146384600F0A6F866
:103420008046B8F1000F00D06FE008204849A1F8AD
:103430000002454800780870434840784870424888
:1034400040880012887040488078C8703E48806884
:10345000007808713C4880684078487106213C48F3
:1034600000F0E2F804463A498C71200AC87144E041
:1034700035484788002517E03348806810F8156004
:10348000314881686800401C085C40EA06263146E5
:10349000384600F06BF88046781C87B2B8F1000F10
:1034A00000D032E0681CC5B227488088A842E3DC1F
:1034B00008202749A1F80002234800780870224814
:1034C0004078487020484088001288701E488078F4
:1034D000C8701D488088001208711B480079487127
:1034E00006211B4800F0A0F8044619498C71200AF7
:1034F000C87102E04FF0010807E000BF00BF1448A8
:10350000B0F8001200F026F8D6E605201049A1F820
:1035100000020D48007808700B48407840F08000A9
:103520004870084680F80280032100F07DF80446C8
:103530000749CC70200A08710846B0F8001200F064
:1035400009F800BFB8E600005C32002064140020D7
:103550006832002070B504460D4603482A462146CD
:10356000C36A984770BD0000E810002070B505469A
:103570000C460026A5F10C000F284AD2DFE800F027
:1035800008090A0B0C1516171821303132333C008C
:1035900000BF00BF00BF00BFA5F10C001E4921F80D
:1035A00010401639086B804733E000BF00BF00BFF2
:1035B000A5F1110019490C54014617480A3044542A
:1035C00027E0211215480E3880F8271080F828408F
:1035D00021121148163880F8241080F8254018E090
:1035E00000BF00BF00BFA5F116010C480B304454CA
:1035F0000948103044540CE0094804840648163841
:1036000044850849486C804703491639086B804750
:1036100000BF00BF304670BDEE11002052000020F8
:103620001C1400204410002030B502464FF6FF70F5
:1036300012E012F8014B6040002308E000F00104A2
:1036400024B14AF2010484EA600000E040101C4604
:103650005D1CABB2082CF1DB0C1EA1F10105A9B277
:10366000E7D130BD00BFFEE710B503461446E018B1
:1036700082B29A4205DD914201DA994207DA0120CD
:1036800010BD914203DB994201DA0120F8E70020E6
:10369000F6E70000154909880144144A11801449CD
:1036A00009880144124A1180124909880144114ACB
:1036B00011800F490988B1F57A7F07D300210C4AA0
:1036C00011800D490988491C0B4A11800949098854
:1036D00042F21072914207D30021064A1180074935
:1036E0000988491C054A1180704700002C00002001
:1036F00032000020340000202E0000203000002086
:10370000002010490880104908801049088010499D
:103710000880084600880F4908800D4800880E4937
:1037200008800B4800880D490880094800880C492A
:103730000880074800880B490880054800880A4926
:103740000880704732000020340000202E00002046
:103750002C00002036000020380000203A00002015
:103760003C0000203E000020400000207047000088
:1037700008B508490968C9084FF47A72B1FBF2F13B
:103780004143009100BF00BF00994A1E00920029EA
:10379000F9D108BD0C0000202DE9F04780460D4608
:1037A0002621404600F0DEF8064616B90020BDE8A6
:1037B000F08740F2B450864200DD0646282140469C
:1037C00000F0D0F80746B946C7F30A0700220121E6
:1037D0003B48FEF7FDF9384600F004F9182101EBEB
:1037E0004811C8B200F0F4F836480068C06800F02C
:1037F000FF0AB819B0F5006F11DA00240CE00020C0
:1038000000F0E6F82F480068C06800F0FF0A85F86D
:1038100000A06D1C601C84B2B442F0DB3BE0C7F535
:10382000006087B200240CE0002000F0D1F82548A9
:103830000068C06800F0FF0A85F800A06D1C601CDD
:1038400084B2BC42F0DB012211461D48FEF7C0F9EC
:10385000002201211A48FEF7BBF9002000F0C2F84F
:10386000182101EB4811C8B200F0B2F81548006801
:10387000C06800F0FF0A0CE0002000F0A9F8114831
:103880000068C06800F0FF0A85F800A06D1C601C8D
:1038900084B2B442F0DB012211460948FEF798F9E0
:1038A00009EB06001FFA80F94A462821404600F03D
:1038B0005BFE40220121404600F036FE304676E7AE
:1038C000000C01407814002070B50446002201214C
:1038D0000D48FEF77DF9204600F084F8012000F045
:1038E00077F80A480068C068C5B2002000F070F898
:1038F00006480068C068C5B2012211460248FEF7BA
:1039000067F9284670BD0000000C014078140020C3
:1039100070B504460D46002201211048FEF758F903
:10392000284600F05FF8082101EB4411C9B241F0CC
:10393000010000F04DF80A480068C068C6B20020D7
:1039400000F046F806480068C068C6B20122114679
:103950000248FEF73DF9304670BD0000000C014002
:103960007814002070B505460E4600220121164845
:10397000FEF72EF9304600F035F8082101EB45112D
:10398000C9B241F0020000F023F810480068C06896
:1039900084B2002000F01CF80C480068C06884B2B3
:1039A000002000F015F84FF6FF7000EA04240748E5
:1039B0000068C068204484B2012211460248FEF724
:1039C00007F9204670BD0000000C0140781400206B
:1039D00001B5FF23012269460148FEF707FE08BD35
:1039E0007814002010B504462012FFF7F1FFE0B272
:1039F000FFF7EEFF10BDF8B504460E4615463346F8
:103A0000012202212046009500F018F828B1606DCF
:103A100040F0200060650320F8BD3346002280217D
:103A20002046009500F00AF828B1606D40F02000B3
:103A300060650320F0E70020EEE700002DE9F84F75
:103A400004460D4690461E46DDF82890FEF7C6F85F
:103A5000A0EB0900371AFEF7C1F882462C4800682F
:103A6000C0F3CB307843009045E0701C002842D072
:103A7000FEF7B4F8A0EB0A00B84200D2A7BB20685A
:103A8000406820F0E000216848606068B0F5827FFF
:103A90000DD1A068B0F5004F03D0A068B0F5806FDD
:103AA00005D12068006820F0400021680860A06A05
:103AB000B0F5005F0DD100BF2068006820F4005011
:103AC000216808602068006840F4005021680860A0
:103AD00000BF012084F8510000BF002084F850008E
:103AE00000BF0320BDE8F88FFFE7009800B900276A
:103AF0000098401E0090206880682840A84201D1AC
:103B0000012000E000204045AFD10020EAE700009E
:103B10000C000020704710B5044601220021204609
:103B200000F002FD01221146204600F0FDFC0520B8
:103B3000FDF7C6FD03212046FFF7EAFE132806D055
:103B400010220121204600F0EFFC002010BD0422CD
:103B50000121204600F0E8FCFF20F7E710B50446FD
:103B600001220021204600F0DFFC01221146204600
:103B700000F0DAFC0520FDF7A3FD03212046FFF746
:103B8000C7FE132806D010220121204600F0CCFCED
:103B9000002010BD02220121204600F0C5FC0520B6
:103BA000FDF78EFD03212046FFF7B2FE142806D054
:103BB00010220121204600F0B7FC0020E9E7FF2099
:103BC000E7E710B5044602220021204600F0ACFCD5
:103BD00001221146204600F0A7FC0520FDF770FDEC
:103BE00003212046FFF794FE222806D0102201214F
:103BF000204600F099FC002010BDFF20FCE70000EB
:103C000010B50120FFF746FD07480121826B904760
:103C100006480121826B904705480121826B90473D
:103C2000FEF71AF810BD0000E81000202C1100204B
:103C30007011002000B58FB0282105A8FCF79DFA6F
:103C400014216846FCF799FA092005904FF480305A
:103C5000069000200790012009900B9002200C9004
:103C6000C1030D914FF4E0110E9105A8FEF7EAF99A
:103C700008B1FDF79BFA0F20009002200190002070
:103C800002904FF480600390002004900221684667
:103C9000FEF7B4F808B1FDF789FA0FB000BD704720
:103CA00010B50848016C88470748016C88470749E8
:103CB000886C8047064948688047064948688047BD
:103CC00010BD0000E81000207011002044100020FA
:103CD0000C140020B41100207047704710B504493F
:103CE000086980470349D1F8D400804710BD00001F
:103CF000C0110020301300207047704710B50249F2
:103D00004868804710BD000098100020704770B5CB
:103D100005466C6A0020E085E0842046FEF7A5FD9C
:103D200070BD70B506460025746A20684069C0F30E
:103D3000C01594F84100212805D125B10020E08468
:103D4000204600F0FBF820684069C0F3801594F825
:103D50004200222805D125B10020E085204600F050
:103D6000A7F8606C40F0100060642046FEF77DFD0F
:103D700070BD70B505466C6A2868006800F02000C8
:103D8000002842D1E08500BF00BF21680C3151E816
:103D9000001F21F4807021680C3141E80002002AE4
:103DA000F3D100BF00BF00BF2168143151E8001FEC
:103DB00021F001002168143141E80002002AF3D10A
:103DC00000BF00BF00BF2168143151E8001F21F07F
:103DD00040002168143141E80002002AF3D100BFFD
:103DE000202084F84200206B01280ED100BF00BFC4
:103DF00021680C3151E8001F21F0100021680C31BE
:103E000041E80002002AF3D100BF00206063206B6C
:103E1000012804D1A18D2046FEF7E1FC02E02046F6
:103E2000FEF7E4FF70BD70B505466C6A0120606363
:103E3000206B012805D1A08D41082046FEF7CFFC5C
:103E400002E02046FEF7D3FF70BD70B505466C6AF0
:103E50002868006800F02000F8B90020E08400BF66
:103E600000BF2168143151E8001F21F08000216853
:103E7000143141E80002002AF3D100BF00BF00BFA7
:103E800021680C3151E8001F41F0400021680C31DD
:103E900041E80002002AF3D102E02046FEF7EEFFDF
:103EA00070BD70B50446656A2846FFF70DF870BD11
:103EB00000BF00BF02680C3252E8002F22F490715C
:103EC00002680C3242E80013002BF3D100BF00BFA0
:103ED00000BF0268143252E8002F22F0010102688C
:103EE000143242E80013002BF3D100BF016B01290B
:103EF0000ED100BF00BF02680C3252E8002F22F042
:103F0000100102680C3242E80013002BF3D100BF0D
:103F1000202180F8421000210163704710B504464B
:103F20002068C06820F040002168C860202084F824
:103F300041002046FEF7A2FF002010BD00BF00BFD9
:103F400002680C3252E8002F22F0C00102680C32E5
:103F500042E80013002BF3D100BF202180F841106C
:103F60007047F8B5044694F84200222875D1A0683D
:103F7000B0F5805F0CD1206950B90025A66A206891
:103F80004068C0F308003080A06A801CA06215E081
:103F9000A56A0026A068B0F5805F03D0A06828B9A4
:103FA000206918B920684068287004E020684068DB
:103FB00000F07F002870A06A401CA062E08D401EC7
:103FC00080B2E085002846D12068C06820F020003B
:103FD0002168C8602068C06820F480702168C860CB
:103FE0002068406920F0010021684861202084F8A1
:103FF000420000206063206B012826D1002020634E
:1040000000BF00BF21680C3151E8001F21F01000F3
:1040100021680C3141E80002002AF3D100BF20687A
:10402000006800F0100010280AD100BF00200090A6
:1040300020680068009020684068009000BF00BFC2
:10404000A18D2046FEF7CBFB02E02046FEF7CEFE18
:104050000020F8BD01E00020FBE70220F9E70000A6
:1040600070B504462168096921F44051E2681143A2
:10407000226811612269A1681143626941EA02055F
:104080002168C96841F20C62914329432268D160DA
:104090002168496921F44071A26911432268516184
:1040A0002D4A2168914202D1FDF784FF01E0FDF71E
:1040B00071FF00EBC00101EB001162689200B1FBDF
:1040C000F2F100EBC00202EB001263689B00B2FB4E
:1040D000F3F26423B2FBF3F202EBC20303EB02122E
:1040E000A1EB8201322202EB01116422B1FBF2F159
:1040F00001F0F00100EBC00202EB001263689B00CC
:10410000B2FBF3F26423B2FBF3F201EB021200EB19
:10411000C00101EB001163689B00B1FBF3F100EB00
:10412000C00303EB00136668B600B3FBF6F3642626
:10413000B3FBF6F303EBC30606EB0313A1EB83011A
:10414000322303EB01116423B1FBF3F101F00F0102
:1041500011442268916070BD0038014077B581B08C
:10416000044615460298A062A585002060642220BE
:1041700084F842002848E16B88622848E16BC862F5
:104180002748E16B08630020E16B486302AE3268A8
:104190002368191D2B46E06BFDF744FA00BF002091
:1041A000009020680068009020684068009000BF80
:1041B00000BF206970B100BF00BF21680C3151E819
:1041C000001F41F4807021680C3141E80002002A90
:1041D000F3D100BF00BF00BF2168143151E8001FB8
:1041E00041F001002168143141E80002002AF3D1B6
:1041F00000BF00BF00BF2168143151E8001F41F02B
:1042000040002168143141E80002002AF3D100BFC8
:10421000002004B070BD0000733D0008273E000878
:10422000233D0008014691F84100212828D18868E3
:10423000B0F5805F0BD1086948B90A6A1088C0F3ED
:1042400008000B685860086A801C086205E00B6A69
:10425000581C086218780B685860C88C401E80B2E1
:10426000C88458B90868C06820F080000B68D8601E
:104270000868C06840F040000B68D86000207047B4
:104280000220FCE708B50D480068006800F0100047
:1042900010280FD100BF0020009008480068006877
:1042A0000090064800684068009000BF00BF0448C6
:1042B000416B88470148FEF7D9FA08BDD0140020A9
:1042C000E810002008B50D480068006800F01000F4
:1042D00010280FD100BF0020009008480068006837
:1042E0000090064800684068009000BF00BF044886
:1042F000416B88470148FEF7B9FA08BD1815002040
:104300007011002000BFFEE710B500221021074801
:10431000FDF75EFC3220FDF7D3F90122102103489E
:10432000FDF756FC6420FDF7CBF910BD00080140F5
:1043300010B500248021002000F0C2F80A20FDF70B
:10434000BFF9042219480168012000F059F904223C
:1043500016480168091D052000F052F9062213488D
:1043600001680831092000F04BF904220F48016868
:104370000E310F2000F044F900BF0BE0E0B2022242
:104380001E2100F0D1F8E0B202221F2100F0CCF88B
:10439000601C84B2082CF1DB4FF4FA61192000F0A4
:1043A000A9F808211B2000F08BF810BD9410002004
:1043B0002DE9F04704460E46904620780021FFF78D
:1043C000A7FA00F00F0022280ED0207804F11B027B
:1043D0000C2100F0E9F894F82030E17F43EA012253
:1043E0002078102100F0C0F820782421FFF7BAFAD5
:1043F0000746B946C7F30A07002201212F48FDF7F7
:10440000E7FB3846FFF7EEFA2178102202EB411164
:10441000C9B241F00400FFF7DBFA07EB0800B0F582
:10442000006F0ADA002505E016F8010BFFF7D0FA55
:10443000681C85B24545F7DB2BE0C7F5006087B205
:10444000002505E016F8010BFFF7C2FA681C85B2DB
:10445000BD42F7DB012211461848FDF7B9FB0022E7
:1044600001211648FDF7B4FB0020FFF7BBFA2178C5
:10447000102202EB4111C9B241F00400FFF7A8FA83
:1044800005E016F8010BFFF7A3FA681C85B2454555
:10449000F7DB012211460948FDF79AFB09EB0800FA
:1044A0001FFA80F920784A46242100F05DF8207830
:1044B0002022012100F038F8BDE8F087000C01400F
:1044C00070B505460C46002201210948FDF780FB26
:1044D0002846FFF787FA0520FFF77AFA2046FFF70C
:1044E00077FA012211460248FDF772FB70BD000009
:1044F000000C014070B505460C4600220121094818
:10450000FDF766FB2846FFF76DFA0620FFF760FA15
:104510002046FFF767FA012211460248FDF758FBD3
:1045200070BD0000000C014070B504460D461646F3
:10453000002201210B48FDF74BFB2846FFF752FAFA
:10454000082101EB4411C9B241F00500FFF740FA20
:104550003046FFF73DFA012211460248FDF738FBCD
:1045600070BD0000000C014070B504460D461646B3
:10457000002201210B48FDF72BFB2846FFF732FAFA
:10458000082101EB4411C9B241F00600FFF720FAFF
:104590003046FFF727FA012211460248FDF718FBC3
:1045A00070BD0000000C014070B505460E46144673
:1045B000002201211148FDF70BFB3046FFF712FAEC
:1045C000082101EB4511C9B241F00700FFF700FADD
:1045D00014F8010BFFF7FCF914F8010BFFF7F8F9D9
:1045E00014F8010BFFF7F4F914F8010BFFF7F0F9D9
:1045F000012211460148FDF7EBFA70BD000C0140A5
:104600002DE9F04107460C461546002201210D48D0
:10461000FDF7DEFA3846FFF7E5F90420FFF7D8F991
:10462000002605E014F8010BFFF7D2F9701C86B2E2
:10463000AE42F7DB012211460248FDF7C9FABDE898
:10464000F0810000000C01400FB4054B10B503A928
:10465000044A029800F068F810BC5DF814FB0000F2
:10466000255B0008681400200FB47CB50C0009AD70
:1046700001D0611E00E00021CDE90001064B6A4631
:104680002946089800F050F8002C02D0009A00212A
:1046900011707CBC5DF814FB7F4B00080FB4084B15
:1046A00010B504A902AA039800F03EF8044602A936
:1046B000002000F06FFA204610BC5DF814FB0000EB
:1046C000954B000802480068C0F3022070470000C4
:1046D0000CED00E010B5002804DB0A07130E054AB4
:1046E000135406E00A07140E034A00F00F031B1FC1
:1046F000D45410BD00E400E018ED00E002E008C86A
:10470000121F08C1002AFAD170477047002001E04B
:1047100001C1121F002AFBD1704730380A2801D28C
:1047200001207047002070472DE9FF4F8DB00F46E4
:104730000546002606E025280BD0DDE90F1290473C
:104740006D1C761C28780028F5D111B03046BDE8E4
:10475000F08F0024A246A1460122E94900E004436B
:1047600015F8013F203B02FA03F00842F7D1287800
:104770002A2810D06FF02F022878A0F130010929E3
:1047800014D80AEB8A0102EB410144F0020400EB69
:10479000010A6D1CF0E701CF5FEA000A03D544F47B
:1047A0000054CAF1000A44F002046D1C28782E2837
:1047B00017D115F8010F44F004042A280ED06FF029
:1047C0002F022878A0F1300109290AD809EB8901C4
:1047D00002EB410100EB01096D1CF2E757F8049B65
:1047E0006D1C28786C280FD006DC4C2817D0682860
:1047F0000DD06A2814D104E0742810D07A280FD183
:104800000DE044F400140AE044F4801401E044F4A0
:1048100040146978814202D104F580146D1C6D1C2E
:1048200028786E281ED00CDC632830D004DC0028E9
:104830008BD0582811D19FE0642867D069280CD10B
:1048400064E073282DD004DC6F2872D0702804D166
:1048500094E075286ED078286DD0DDE90F1290476E
:10486000761C4BE1C4F30250022806D0032809D07D
:10487000042801CF09D0066040E101CFF117C0E95B
:1048800000613BE101CF068038E1067036E117F8A0
:10489000040B8DF8000000208DF80100EB4601208C
:1048A00003E057F804BB4FF0FF3061074FF0000101
:1048B00002D40DE008F10101884649450FDA804530
:1048C000F8DB1BF808100029F4D108E008F1010119
:1048D00088468142FADB1BF808100029F6D1DDE991
:1048E0000F23AAEB08008146214600F031F930443D
:1048F00000EB080604E0DDE90F121BF8010B9047FE
:10490000B8F10108F7D221464846F2E00A21C4F383
:1049100002524FF0000B0891022A04D001CFC117B8
:10492000032A09D00AE0FF1D27F00707F7E8020174
:1049300008E02CE01EE01FE000B2C117042A01D1FC
:1049400040B2C117021E71F1000206DA0023D0EB5B
:10495000030063EB01012D2202E0220504D52B2286
:104960008DF82420012203E0E20701D02022F7E79E
:10497000904653E00A210BE0102109E010214FF08E
:10498000000B44F004044FF00809089103E00821EB
:104990004FF0000B0891C4F30252022A04D001CF59
:1049A0000021032A06D006E0FF1D27F00707F7E8DD
:1049B000020103E080B2042A00D1C0B24FF0000827
:1049C00022072BD52A78702A07D0DDF820C08CF07A
:1049D000100C5CEA0B0C05D00EE040228DF8242070
:1049E000012208E050EA010306D030238DF824307C
:1049F0008DF8252002229046089B83F0080353EA95
:104A00000B030BD150EA010201D1620706D5302217
:104A10008DF824204FF00108A9F101092A78582ABD
:104A200004D038A20B9208AA0A920BE03AA2F9E746
:104A30005B46089AFBF742FE0B9B9B5C0A9A521E50
:104A40000A92137050EA0102F2D10A98ADEB00000D
:104A500000F1200B600702D524F4803401E04FF010
:104A60000109D94502DDA9EB0B0000E0002000EBB5
:104A70000B0141440890AAEB010AE00306D4DDE9EA
:104A80000F232146504600F063F806444FF000091A
:104A900008E009A911F80900DDE90F12904709F1B2
:104AA0000109761CC145F4DBE0030CD5DDE90F23D9
:104AB0002146504600F04CF8064404E0DDE90F12B0
:104AC00030209047761C0899481E08900029F5DC94
:104AD00008E00A980A990078491C0A91DDE90F124A
:104AE0009047761CBBF10001ABF1010BF1DC2146D4
:104AF0005046DDE90F2300F019F806446D1C21E64D
:104B000009280100303132333435363738396162A3
:104B10006364656600000000303132333435363767
:104B20003839414243444546000000002DE9F04138
:104B3000044600251E461746880404D405E039467D
:104B40002020B0476D1C641EF9D52846BDE8F081D1
:104B50002DE9F041044600251E469046C80301D5C4
:104B6000302700E02027880404D505E04146384678
:104B7000B0476D1C641EF9D52846BDE8F0814A682F
:104B8000002A06D00A68531C0B6010704868401E4B
:104B9000486070470A68531C0B6010707047000033
:104BA0001FB5402000900020019002900320039048
:104BB00069460248FCF76AFE1FBD0000000C014078
:104BC0001FB540200090112001900020029003208A
:104BD000039069460148FCF759FE1FBD000C0140D7
:104BE00010B5012280212148FCF7F2FF002220218C
:104BF0001E48FCF7EDFF00F09FF81D480068008894
:104C0000632818DC1A48006880780C2813DC1848E0
:104C10000068C0781F280EDC154800680079172846
:104C200009DC1348006840793B2804DC1048006820
:104C300080793B2818DD19200D490968088001207A
:104C40000B49096888700A490968C870002008493A
:104C50000968087106490968487105490968887139
:104C60000348006800F006F810BD0000000C014089
:104C7000D411002070B504462E48006800886328CF
:104C800018DC2C48006880780C2813DC2948006860
:104C9000C0781F280EDC274800680079172809DC37
:104CA0002448006840793B2804DC22480068807969
:104CB0003B2801DD002070BD00218E2000F00AFAA3
:104CC0008021084600F006FA2078FEF700F9054634
:104CD00029468C2000F0FEF9A078FEF7F8F805468A
:104CE0002946882000F0F6F9E078FEF7F0F805464E
:104CF0002946862000F0EEF92079FEF7E8F805460F
:104D00002946842000F0E6F96079FEF7E0F80546D0
:104D10002946822000F0DEF9A079FEF7D8F8054692
:104D20002946802000F0D6F980218E2000F0D2F9AB
:104D30000120C0E7D411002010B58C2000F08AF8C3
:104D400004462046E21704EB12721211A4EB021281
:104D50002146E31704EB13731B1103EB830302EBF0
:104D600043023B4B1B681A80882000F073F804460E
:104D70002046E21704EB12721211A4EB0212214634
:104D8000E31704EB13731B1103EB830302EB4302E2
:104D90002F4B1B689A70862000F05CF80446204672
:104DA000E21704EB12721211A4EB02122146E31770
:104DB00004EB13731B1103EB830302EB4302244B3D
:104DC0001B68DA70842000F045F804462046E2179C
:104DD00004EB12721211A4EB02122146E31704EB4A
:104DE00013731B1103EB830302EB4302184B1B6885
:104DF0001A71822000F02EF804462046E21704EBD8
:104E000012721211A4EB02122146E31704EB137382
:104E10001B1103EB830302EB43020D4B1B685A711A
:104E2000802000F017F804462046E21704EB1272C7
:104E30001211A4EB02122146E31704EB13731B11AA
:104E400003EB830302EB4302014B1B689A7110BD15
:104E5000D411002070B50546012280219C48FCF742
:104E6000B7FE00BF00BF00BF00BF00BF00BF00BF54
:104E700000BF00BF00BF00BF00BF00BF00BF00BF3A
:104E800000BF00BF00BF00BF00BF00BF00BF00BF2A
:104E900000BF00BF00BF00BF00BF00BF00BF45F0A4
:104EA0000105002474E005F0010028B10122402131
:104EB0008748FCF78DFE04E0002240218448FCF77F
:104EC00087FE00BF00BF00BF00BF00BF00BF00BF24
:104ED00000BF00BF00BF00BF00BF00BF00BF00BFDA
:104EE00000BF00BF00BF00BF00BF00BF00BF00BFCA
:104EF00000BF00BF00BF00BF00BF00BF00BF012256
:104F000020217348FCF764FE00BF00BF00BF00BF54
:104F100000BF00BF00BF00BF00BF00BF00BF00BF99
:104F200000BF00BF00BF00BF00BF00BF00BF00BF89
:104F300000BF00BF00BF00BF00BF00BF00BF00BF79
:104F400000BF00BF002220216148FCF741FE00BFE6
:104F500000BF00BF00BF00BF00BF00BF00BF00BF59
:104F600000BF00BF00BF00BF00BF00BF00BF00BF49
:104F700000BF00BF00BF00BF00BF00BF00BF00BF39
:104F800000BF00BF00BF00BF00BF6D10601CC4B2F7
:104F9000082C88DBFFF704FE002470E07610402127
:104FA0004B48FCF703FE10B146F0800601E006F026
:104FB0007F0600BF00BF00BF00BF00BF00BF00BF33
:104FC00000BF00BF00BF00BF00BF00BF00BF00BFE9
:104FD00000BF00BF00BF00BF00BF00BF00BF00BFD9
:104FE00000BF00BF00BF00BF00BF00BF00BF012265
:104FF00020213748FCF7ECFD00BF00BF00BF00BF19
:1050000000BF00BF00BF00BF00BF00BF00BF00BFA8
:1050100000BF00BF00BF00BF00BF00BF00BF00BF98
:1050200000BF00BF00BF00BF00BF00BF00BF00BF88
:1050300000BF00BF002220212548FCF7C9FD00BFAA
:1050400000BF00BF00BF00BF00BF00BF00BF00BF68
:1050500000BF00BF00BF00BF00BF00BF00BF00BF58
:1050600000BF00BF00BF00BF00BF00BF00BF00BF48
:1050700000BF00BF00BF00BF00BF601CC4B2082C4F
:105080008CDB002280211248FCF7A2FD00BF00BF8C
:1050900000BF00BF00BF00BF00BF00BF00BF00BF18
:1050A00000BF00BF00BF00BF00BF00BF00BF00BF08
:1050B00000BF00BF00BF00BF00BF00BF00BF00BFF8
:1050C00000BF00BF00BF00BFFFF77AFD304670BDD4
:1050D000000C014070B505460E46012280219C4817
:1050E000FCF776FD00BF00BF00BF00BF00BF00BFE0
:1050F00000BF00BF00BF00BF00BF00BF00BF00BFB8
:1051000000BF00BF00BF00BF00BF00BF00BF00BFA7
:1051100000BF00BF00BF00BF00BF00BF00BF00BF97
:1051200005F0FE05002474E005F0010028B101221D
:1051300040218748FCF74CFD04E0002240218448D0
:10514000FCF746FD00BF00BF00BF00BF00BF00BFAF
:1051500000BF00BF00BF00BF00BF00BF00BF00BF57
:1051600000BF00BF00BF00BF00BF00BF00BF00BF47
:1051700000BF00BF00BF00BF00BF00BF00BF00BF37
:10518000012220217248FCF723FD00BF00BF00BFB1
:1051900000BF00BF00BF00BF00BF00BF00BF00BF17
:1051A00000BF00BF00BF00BF00BF00BF00BF00BF07
:1051B00000BF00BF00BF00BF00BF00BF00BF00BFF7
:1051C00000BF00BF00BF002220216148FCF700FDA6
:1051D00000BF00BF00BF00BF00BF00BF00BF00BFD7
:1051E00000BF00BF00BF00BF00BF00BF00BF00BFC7
:1051F00000BF00BF00BF00BF00BF00BF00BF00BFB7
:1052000000BF00BF00BF00BF00BF00BF6D10601C2B
:10521000C4B2082C88DB002474E006F0010028B139
:10522000012240214A48FCF7D3FC04E0002240213F
:105230004748FCF7CDFC00BF00BF00BF00BF00BF68
:1052400000BF00BF00BF00BF00BF00BF00BF00BF66
:1052500000BF00BF00BF00BF00BF00BF00BF00BF56
:1052600000BF00BF00BF00BF00BF00BF00BF00BF46
:1052700000BF012220213648FCF7AAFC00BF00BF76
:1052800000BF00BF00BF00BF00BF00BF00BF00BF26
:1052900000BF00BF00BF00BF00BF00BF00BF00BF16
:1052A00000BF00BF00BF00BF00BF00BF00BF00BF06
:1052B00000BF00BF00BF00BF002220212448FCF730
:1052C00087FC00BF00BF00BF00BF00BF00BF00BF22
:1052D00000BF00BF00BF00BF00BF00BF00BF00BFD6
:1052E00000BF00BF00BF00BF00BF00BF00BF00BFC6
:1052F00000BF00BF00BF00BF00BF00BF00BF7610EF
:10530000601CC4B2082C88DB002280211048FCF706
:105310005FFC00BF00BF00BF00BF00BF00BF00BFF9
:1053200000BF00BF00BF00BF00BF00BF00BF00BF85
:1053300000BF00BF00BF00BF00BF00BF00BF00BF75
:1053400000BF00BF00BF00BF00BF00BF00BF70BDF7
:10535000000C014010B586B0044600200190029078
:1053600004940120059001A902A8FCF7BDF906B03C
:1053700010BD000010B5064948688047162205494F
:10538000054800F0B5F802494868804710BD0000A4
:10539000B4110020EE11002000FC000810B5162208
:1053A0000E49A1F11600FAF7FAFEA8B10C494868B7
:1053B000804772B6162209490A4800F0BDF8044633
:1053C0002CB916220549A1F11600FAF7BDFE62B606
:1053D00003494868804700BF10BD0000EE1100205F
:1053E000B411002000FC000810B541F28834C0213F
:1053F0000F4880F82010A82180F82110012180F8A2
:105400002210652180F82310211280F8241080F8E2
:105410002440FF2180F8261080F8271080F82810FB
:10542000002180F829100A214185FFF7B7FF10BD40
:10543000D811002010B5FFF79DFF2A4890F82000F2
:10544000FF2810D1274890F82100FF280BD12548CC
:1054500090F82200FF2806D1224890F82300FF2868
:1054600001D1FFF7C1FF16221E4916311D48FAF778
:105470006BFE1C4890F820001B498873194890F86F
:1054800021101948C173174890F82210164801746A
:10549000144890F8231014484174124890F82410CE
:1054A000114880F827100F4890F825100E4880F812
:1054B00028100C4890F826100B484176094890F8BF
:1054C000271009488176074890F828100648C176C9
:1054D000044890F82910044801770248408D034998
:1054E000088410BDD8110020440000201C140020A6
:1054F0002DE9F84103460C4621461D46960802F068
:105500000307002005E055F820C0C1F800C0091DC0
:10551000401CB042F7D36FB155F826000090EC461E
:10552000002004E01CF8008001F80080401CB84214
:10553000F8D300BFBDE8F8812DE9FC5F0746884637
:10554000154600244646A808019005F00309BA460E
:10555000FCF784F93846FFF7FDFE044624B1FCF75A
:105560001BF92046BDE8FC9F4FF0000B0FE0D6F87A
:1055700000C06246002351460220FCF717F904469A
:1055800004B107E00AF1040A361D0BF1010B019882
:105590008345ECD300BFB4B9B9F1000F13D04FF07D
:1055A000FF300090EB46002003E0315C0BF8001068
:1055B000401C4845F9D3002351460220009AFCF7CD
:1055C000F5F8044600BFFCF7E7F82046CAE70000FC
:1055D00010B54FF400410448FCF7F0FA4FF40051C5
:1055E0000248FCF7EBFA10BD000801400010014032
:1055F00010B500240EE03220FBF76AFD4FF40041A5
:105600000648FCF7DBFA4FF400510548FCF7D6FAE0
:10561000601CC4B2142CEEDB10BD00000008014079
:105620000010014070B504460E46154600BFA07C30
:105630000028FCD00020A074A08BA84200DAA58B23
:105640002A4631466069FAF77FFD2A46616960683B
:10565000FDF7CEFB70BD10B5044660680068C068F9
:1056600040F0100061680968C860E28BA169606859
:10567000FDF7A6FB10BD70B504466068FDF7B0F8F5
:10568000E08BE16809684968401A86B206B970BDC6
:10569000002506E0A2695119206801F0F4FF681C9A
:1056A00085B2B542F6DB204600F040F8E28BA169F6
:1056B0006068FDF785FB00BFE9E7000070B50446B0
:1056C000A08C618C884225DA20688089208420465D
:1056D00000F032F8208CE18B88421BDC208CC8B1B2
:1056E000208CB0F5007F03D9206801F080FF11E025
:1056F000002506E0084A5119206801F080FF681C67
:1057000085B2208CA842F5DCE06B18B1218C0248F0
:10571000E26B904770BD0000901A002090F82620A0
:10572000012A02D1428C0A4442847047012180F848
:105730002610002141847047002180F82610418402
:1057400070472DE9F04104460F461646A08B96FBA4
:10575000F0F01FFA80F8002507E0A28B02FB05712C
:105760002046FFF75FFF681C85B24545F5DBA08B3F
:1057700000FB156086B20EB9BDE8F081A08B00FB7E
:10578000057132462046FFF74DFF00BFF4E70121C7
:105790008174704710B5FEF7B7FDFEF7C9FDFBF742
:1057A0009DFC002416E040F20B4161430B4A126855
:1057B000143202EB810000F0D3F8002240F20B40DB
:1057C000604306490968143101EB800080F822200B
:1057D000601CC4B2012CE6DB10BD00009410002058
:1057E00070B500BF1720FEF76FF806460A20FBF7DA
:1057F00067FF0024A9E00120A040304000287DD0B0
:1058000040F20B416143554A1268143212F82100EC
:105810000221FEF77DF8054640F20B4161434F4AF5
:105820001268143212F821002A460221FEF77CFE8B
:1058300005F00100A8B140F20B40604347490968F8
:10584000143101EB800090F8220040F0020240F297
:105850000B40604341490968143101EB800080F836
:10586000222005F0020000B340F20B4161433B4AA5
:105870001268143212F8210010220121FEF754FEA2
:1058800040F20B416143354A1268143202EB810049
:1058900000F066F8002240F20B4060432F4909688F
:1058A000143101EB800080F8222005F01000A8B12F
:1058B00040F20B40604329490968143101EB800034
:1058C00090F8230040F0020240F20B40604323496D
:1058D0000968143101EB800080F8232005F00400F2
:1058E000B8B140F20B4060431C490968143101EB28
:1058F000800090F8230040F0010200E023E040F235
:105900000B40604315490968143101EB800080F8B1
:10591000232005F00800B0B140F20B4161430F4A6B
:105920001268143212F8210010220121FEF7FCFD4A
:10593000002240F20B40604308490968143101EB32
:10594000800080F82320601CC4B2012CFFF653AF06
:105950001720FDF7B9FF00B144E770BD9410002097
:1059600010B50446207840F2B4521221FEF7FCFD37
:10597000237DE17C43EA012220780421FEF7F4FD37
:10598000A37E617E43EA012220781021FEF7ECFD20
:10599000207804F115020C21FEF706FE10BD10B5AB
:1059A000044694F8220080BB94F8210020B101281D
:1059B0000FD0022827D119E02078FEF7CFF8FF2872
:1059C00003D1012084F8220002E0002084F82200A4
:1059D0001AE02078FEF79FF8FF2803D1012084F811
:1059E000220002E0002084F822000DE02078FEF77B
:1059F000E8F8FF2803D1032084F8220002E0002009
:105A000084F8220000E000BF00BF10BD70B5002484
:105A10000BE040F20B416143384A1268143202EB4A
:105A20008100FFF7BCFF601CC4B2012CF1DBFFF763
:105A3000D7FE00245FE040F20B4060432F49096825
:105A4000143101EB800090F8230000F001000028E1
:105A50004FD040F20B40604328490968143101EBF4
:105A6000800090F8230020F0010240F20B406043D8
:105A700022490968143101EB800080F8232040F2AC
:105A80000B4060431D4A1268143202EB800000F1A3
:105A900024010020FDF780FE054640F20B406043E4
:105AA00016490968143101EB800000F58050806AC6
:105AB000F0B140F20B426243104E3668143606EBEA
:105AC000820202F1240140F20B4262430B4E36681F
:105AD000143606EB820040F20B426243074E3668F2
:105AE000143606EB820202F58052936A2A469847E2
:105AF00000BF601CC4B2012C9DDB70BD941000205F
:105B000010B50248FCF7A1F810BD00006C1400208D
:105B10000348406840F480700149486070470000C5
:105B2000002004E038B504460D46E0B2009003487A
:105B300001226946C36A984738BD0000E81000207A
:105B4000FCF796F8FEF776F8FDF700FAFDF7CCF9CA
:105B5000FDF7A8FAFDF7C8FAFDF7E2FAFDF78EFAAD
:105B6000FBF7BCF904E0FBF7F9F90248FCF76DF824
:105B7000F9E700006C14002070B503460C4603E002
:105B800014F8015B03F8015B151EA2F10102F7D1C5
:105B900070BD2DE9F04105460E464FF0000837680C
:105BA0007079012101EB8000287070791A283DD0AE
:105BB00011DC112829D007DCF0B1082823D00928EE
:105BC00022D0102861D127E0122830D018284ED0DA
:105BD00019285AD11BE0282847D006DC1C2836D0CB
:105BE000202843D0242850D130E029280ED02A285C
:105BF0001BD02C2849D128E04FF00208F0796870BA
:105C00004046BDE8F08100BF00BF00BF00BF38784C
:105C1000A8704FF0030838E0F2793946A81CFAF76B
:105C200093FAF07900F102082FE000BF00BF0024D2
:105C300006E0C4F10100395CA01C2954601CC4B208
:105C4000022CF6DB4FF004081FE000BF00BF002469
:105C500006E0C4F10300395CA01C2954601CC4B2E6
:105C6000042CF6DB4FF006080FE000BF00BF002455
:105C700006E0C4F10700395CA01C2954601CC4B2C2
:105C8000082CF6DB4FF00A0800BF00BFA8F10200A5
:105C900068704046B5E770B504460D4600212846B9
:105CA00001F075FD20600021281D01F051FDA0804C
:105CB000A879A071E879E071287A2072687A607218
:105CC000002105F10A0001F062FDE06070BD0000F6
:105CD0000149024881627047DD75000858100020B4
:105CE00070B505460C460E2C00DA70BD29464548B5
:105CF0000068FFF7D0FF434800680068001DA0421D
:105D000000D0F2E73F480068007A00B1EDE73D4877
:105D10000068407A0A2871D2DFE800F005213A3B9A
:105D200053546C6E706F37480068008C35490968B1
:105D30008988884200D0D8E73248006831490E6827
:105D40004ECE10304EC0A4F10E0082B22E4805F1A6
:105D50000E0103682B480068103098474FE029482F
:105D6000006828490B68D3E901621968DB68C0E95B
:105D70000562C36101610221224800684176002367
:105D80001A4619461F480068103000F051F836E0F6
:105D900035E01C4802680668D6E901313068F668CB
:105DA000C2E90616C2E904030421164800684176D8
:105DB00000231A46194613480068103000F038F8DE
:105DC0001DE01CE00F4801680668D6E9010332684F
:105DD000F668C1E90636C1E90420062109480068D1
:105DE000417600231A46194606480068103000F034
:105DF0001FF804E003E001E001E000E000BF00BFA5
:105E000000BF72E7481400200C14002070B504464F
:105E10000D4629462046FBF75AF904482A462146F2
:105E2000C36CA0F6EC70984770BD000044100020D1
:105E30002DE9F0470446884616469946184D06F166
:105E40000A00206000222946206801F064FCA08836
:105E50000022291D01F042FCA079A871E079E871C7
:105E6000207A2872607A6872002205F10A01E068DF
:105E700001F051FC0E27B8F1000F07D036B1E81938
:105E800032464146FAF760F9B81987B239462846D2
:105E9000FFF7BCFF39462846FBF719F9BDE8F08744
:105EA0005C2E002001480249C8637047A5320008F3
:105EB000E8100020704700000748D0F8B00000212B
:105EC000054AD2F8B4200B4611431843034A12681E
:105ED00042F8901F506070473013002008140020D3
:105EE00010B502460B460020002104E0545C044437
:105EF000E0B24C1CA1B29942F8DB10BD0EB50320F4
:105F00008DF80000034909680868694601F0BBFB89
:105F10000EBD0000081400203EB5044604208DF894
:105F200000008DF80240034909680868694601F0DD
:105F3000AAFB3EBD08140020FEB504460D461646D9
:105F400005208DF800008DF801408DF80250ADF865
:105F50000460034909680868694601F094FBFEBDC6
:105F6000081400203EB5044600208DF800008DF88E
:105F70000140034909680868694601F084FB3EBD99
:105F8000081400203EB5044602208DF800008DF86C
:105F90000140034909680868694601F074FB3EBD89
:105FA000081400200448018804480068A0F89810EC
:105FB00003480449C86370472C00002008140020DF
:105FC000C95F0008701100202DE9F04786B0044633
:105FD0000E462078022802D006B0BDE8F087301FB8
:105FE000205C032803D1701E205C0D2800D0F3E74D
:105FF000A74800680079062817D0F01E81B2204615
:10600000FFF76EFF07463A46A2A105A8FEF746FB3A
:106010009DF81410F01E205C814205D19DF81510EA
:10602000B01E205C814200D0D6E74FF00008651C0E
:10603000974800680079082872D2DFE800F004F180
:1060400005060708165F00BF00BF00BF00BF0222A1
:1060500092A12846FAF7B0F820B94FF0010800F0F5
:1060600037F901E04FF00008DBE00027A14688483F
:10607000006800F1080A28E0781C04EB00094B4690
:1060800087A2032102A8FEF7EFFA01AA85A102A8C0
:10609000FAF7A2F80198162803DD07F10E0087B27F
:1060A00013E009F103037EA2082102A8FEF7DCFA3F
:1060B0006A467DA102A8FAF78FF8DDE900014AF8E7
:1060C000210007F10E0087B200BFB742D4DBA7F171
:1060D0000E0087B2781C04EB0009032273A1484626
:1060E000FAF76AF838B94FF00108012168480068EA
:1060F00080F8891001E04FF0000892E003226CA1C3
:106100002846FAF759F810B14FF0000889E0E8780E
:106110004E2806D100205E49096881F8AC000CE0E9
:106120007EE0E878532805D101205949096881F8B3
:10613000AC0002E04FF0000873E02879522805D146
:1061400000215348006880F8AD100BE028795328EF
:1061500005D101214E48006880F8AD1002E04FF0F3
:1061600000085EE06879522805D10021484800689F
:1061700080F8AE100BE06879532805D1012144481E
:10618000006880F8AE1002E04FF0000849E00021FE
:106190003F480068C0F8B0103D480068C0F8B4102F
:1061A000002731E0B81D43193DA2022102A8FEF7E5
:1061B0005BFA01AA3FA102A8FAF70EF8344800687A
:1061C000D0F8B000019901F00F0108433049096887
:1061D000C1F8B00007F10E00431931A2022102A854
:1061E000FEF742FA01AA33A102A8F9F7F5FF284801
:1061F0000068D0F8B400019901F00F010843244968
:106200000968C1F8B4007F1C082FCBD300F060F8F8
:1062100018B906201E49096808714FF0010800E00E
:1062200000BF00BF1A4800680079062825D1184829
:10623000006890F88800012827D11548006890F878
:106240008900012810D100201149096881F88800CF
:1062500000210F48006880F889100D480068A0F8F8
:106260008A1000F035F810E0B8F1000F0DD00021D1
:1062700007480068A0F88A1007E0B8F1000F04D0C2
:106280000020034909684871A6E600BFA4E60000A3
:106290000814002025303258000000004F4B000049
:1062A000257300002564000025660000454E44006B
:1062B0004D3231002575000070B504460D46034887
:1062C0002A462146C36A984770BD0000701100201D
:1062D0000EB50D4909680868694601F090F928B9BA
:1062E000072009490968087100200EBD9DF80000CB
:1062F0000549096808710448006880309DE80E006F
:1063000020300EC00120F0E708140020F0B587B05F
:1063100005461C4D02208DF808001BA21BA10DF1A3
:106320000900FEF7BBF9002412E0C4F10700800069
:1063300025FA00F000F00F000DF804001DF804200D
:10634000211D02ABC81812A1FEF7A8F9601CC4B247
:10635000082CEADB03208DF814000D2102A8FFF7BA
:10636000BFFD07463A460BA10DF11500FEF796F961
:106370000D208DF817001026314602A8FFF79CFF6C
:1063800007B0F0BDFFD97F004D323000257300000B
:1063900025580000253032580000000030B585B087
:1063A00002208DF800000FA20FA10DF10100FEF7F1
:1063B00075F903208DF8040005216846FFF790FD6C
:1063C00005462A4609A10DF10500FEF767F90D20E3
:1063D0008DF80700082421466846FFF76DFF05B0D9
:1063E00030BD00004D323100257300002530325899
:1063F0000000000030B585B002208DF800000FA22B
:106400000FA10DF10100FEF749F903208DF80400FA
:1064100005216846FFF764FD05462A4609A10DF1EE
:106420000500FEF73BF90D208DF8070008242146F2
:106430006846FFF741FF05B030BD0000533232001F
:1064400025730000253032580000000070B586B07A
:10645000044602208DF8040015A216A10DF10500D6
:10646000FEF71CF91CB94E208DF8080007E0012C3E
:1064700003D153208DF8080001E006B070BD032061
:106480008DF80900062101A8FFF72AFD06463246CD
:1064900009A10DF10A00FEF701F90D208DF80C009D
:1064A0000925294601A8FFF707FF00BFE5E700001F
:1064B00053323300257300002530325800000000AD
:1064C0002DE9F04186B004460D46164602208DF8AF
:1064D000040021A221A10DF10500FEF7DFF81CB98F
:1064E0004D208DF8080008E0012C03D142208DF8E2
:1064F000080002E006B0BDE8F0811DB94E208DF81D
:10650000090006E0012D03D153208DF8090000E0B9
:10651000F0E742F2AC60864200DD6326324610A10D
:106520000DF10A00FEF7BAF803208DF80C000921DE
:1065300001A8FFF7D5FC804642460AA10DF10D00E7
:10654000FEF7ACF80D208DF80F000C27394601A896
:10655000FFF7B2FE00BFCDE75332340025730000D1
:1065600025640000253032580000000070B586B068
:10657000044602208DF8040015A216A10DF10500B5
:10658000FEF78CF81CB94D208DF8080007E0012CAF
:1065900003D142208DF8080001E006B070BD032051
:1065A0008DF80900062101A8FFF79AFC064632463D
:1065B00009A10DF10A00FEF771F80D208DF80C000D
:1065C0000925294601A8FFF777FE00BFE5E700008F
:1065D000533230002573000025303258000000008F
:1065E00070B586B0044602208DF8040015A216A1ED
:1065F0000DF10500FEF752F81CB94D208DF808008A
:1066000007E0012C03D142208DF8080001E006B01C
:1066100070BD03208DF80900062101A8FFF760FC7A
:106620000646324609A10DF10A00FEF737F80D20A3
:106630008DF80C000925294601A8FFF73DFE00BF93
:10664000E5E7000053323100257300002530325851
:106650000000000010B500244548006890F888004C
:10666000012828D14248006890F88900012822D0EA
:106670003F480068B0F88A00401C81B23C4800687E
:10668000A0F88A103A480068B0F88A00032811DBA5
:1066900000203749096881F88800002134480068E3
:1066A00080F8891032480068A0F88A100720304925
:1066B0000968087110BD2E480068007908283DD28D
:1066C000DFE800F0043C0B12151C2B382849096840
:1066D00091F8A100FFF74AFF31E02549096891F8D8
:1066E000A100FFF77DFF2AE0FFF784FE27E02049A5
:1066F000096891F8A200FFF7A9FE20E01C4B1B6877
:10670000B3F8A4201A4B1B6893F8A210184B1B680F
:1067100093F8A100FFF7D4FE11E015490968D1F8FC
:10672000A800FFF7F3FD01201149096881F88800EE
:10673000012404E0FFF732FE012400E000BF00BFA7
:1067400004B1B7E70A4800684079401C0849096865
:106750004871074800684079032807DB0020044996
:1067600009684871072002490968087100BFA1E75C
:10677000081400202DE9F047074689464FF0000A2B
:10678000D0460025387800F00300012802D0002010
:10679000BDE8F08738788010854948712DE00AF10E
:1067A000010000F0FF0A785D00F00300012801D02D
:1067B0000020EDE7785D801010B9A81C85B21CE0C0
:1067C000785D80107A4901EBC8014871681C85B278
:1067D000785D774901EBC8018871681C85B278192A
:1067E000734941F83800084600EBC8008079284416
:1067F00085B208F1010000F0FF08A9F10100A842EC
:10680000CDDC00250024CDE0694800EBC4004079D0
:106810001A2847D010DC112821D006DC08281CD00B
:1068200009281BD010283BD11CE012283BD0182887
:106830007ED01928F7D114E028287AD006DC1C284D
:1068400059D0202876D02428EDD153E0292807D02C
:106850002A2826D02C28E6D14BE000BF00BF00BF7D
:1068600000BF00BF524B03EBC4039A79504B53F85F
:106870003410504B5819F9F767FC4D4800EBC40031
:1068800080794B4901EBC401C8714A482844484902
:1068900041F83400084600EBC4008079284485B2F2
:1068A0007DE000BF00BF424951F83400002607E0F8
:1068B000C6F10101415CAA193E4B9954711CCEB23C
:1068C000022EF5DB3A4A02EBC402917901EBD17258
:1068D0005210374B03EBC403DA7136492944344A6A
:1068E00042F83410114601EBC401897929448DB274
:1068F00055E000BF00BF2E4850F83410002607E0D6
:10690000C6F10300085CAA192A4B9854701CC6B241
:10691000042EF5DB264A02EBC4029079C21700EB85
:1069200092729210224B03EBC403DA71214802E009
:106930000EE00BE00BE028441D4A42F834001046FC
:1069400000EBC4008079284485B228E000BF00BF76
:10695000174850F83410002607E0C6F10800085C1C
:10696000AA19144B9854701CC6B2082EF5DB104AB5
:1069700002EBC4029079C21700EB5272D2100C4B9A
:1069800003EBC403DA710B482844094A42F8340087
:10699000104600EBC4008079284485B200BF00BFD8
:1069A000601CC4B24445FFF62FAF4046F0E600003D
:1069B000082B0020982C00202DE9F04F85B00646CA
:1069C00088469146F079B17901F07F0140EA0120D3
:1069D0000490B0790121B1EBD01F07D040F20251F1
:1069E0000498884202D005B0BDE8F08F4946404681
:1069F000FFF7C0FE039040F21F220498811A9042D4
:106A000075D008DCA0F20110002871D0022809D04E
:106A10000C286ED138E112296CD0A1F2E3210029B3
:106A2000F7D122E1CE4840792C287AD10227CC48F0
:106A300004682068B0F1FF3F07D14FF6FF730022D2
:106A40001146304600F0DAFACDE720681F2804D955
:106A500040F6B9312068884204D340F6BC31206842
:106A6000884200D9BFE720681F280BD8BD4D206899
:106A700055F8200002900123242202A9304600F09C
:106A8000BDFA6DE040F6B9312068884219D1B548A9
:106A9000083890F8AC0010B94E2001900AE0B148D7
:106AA000083890F8AC00012802D15320019001E091
:106AB000002001900123102201A9304600F09EFA27
:106AC0004EE040F6BA31206888421DD1A54808380A
:106AD00090F8AD0010B9522001900EE0A14808389E
:106AE00090F8AD00012806D15320019005E0D1E0D7
:106AF000B5E031E136E0002001900123102201A928
:106B0000304600F07BFA2BE040F6BB31206888422B
:106B10001AD19448083890F8AE0018B95220019064
:106B20000BE01EE08F48083890F8AE00012802D133
:106B30005320019001E0002001900123102201A9BF
:106B4000304600F05BFA0BE040F6BC31206888422A
:106B500006D100BF01232C2201A9304600F04EFAD5
:106B600000BFFAE07E4805682B467FA204216846F4
:106B7000FDF77AFD03227DA16846F9F71DFB08B9F0
:106B800000241EE003227AA16846F9F715FB08B934
:106B9000022416E0032277A16846F9F70DFB08B935
:106BA00003240EE0032274A16846F9F705FB08B937
:106BB000042406E0032271A16846F9F7FDFA00B942
:106BC00005246748856828784D2802D14FF0000ACF
:106BD00004E02878422801D14FF0010A6048056995
:106BE00028784E2801D1002703E02878532800D1C7
:106BF00001275B488569B5F800B0062C28D2DFE88C
:106C000004F003270A11171E56480838D0F8B810A8
:106C1000504688471CE053480838D0F8BC1050460E
:106C2000884715E04F490839D1F8C00080470FE088
:106C30004C480838D0F8C4103846884708E049481E
:106C400008385A463946D0F8C8305046984700BFF1
:106C500000BF00221146304600F0B0FB7DE000226C
:106C60001146304600F000F977E03D4840790828A9
:106C700009D13B480468207820B93A490839D1F84D
:106C80009C00804700BF68E000221146304600F0BB
:106C900043F962E03248407910285CD130480468FA
:106CA000207830384FF47A7148436178303901EBFD
:106CB000C10202EB011100EB8101A078303800EB3A
:106CC000800001EB4001E0783038084480B2ADF834
:106CD0000400607930382179303901EB810100EB13
:106CE0004100C0B28DF80600E0793038A179303922
:106CF00001EB810100EB4100C0B28DF80700E079A3
:106D00003038A179303901EB810100EB4100C0B28C
:106D10008DF80800E0793038A179303901EB810134
:106D200000EB4100C0B28DF80900607A3038217A5A
:106D3000303901EB810100EB4100C0B28DF80A004F
:106D40000F48C16801A8884720B10022114630468B
:106D500000F00CFB00BF00E000BF00BF00BF42E638
:106D6000082B002038130020257300005332300018
:106D70005332310053323200533233005332340035
:106D8000C01100202DE9F04104460D461646044886
:106D9000002332462946876A2046B847BDE8F0817D
:106DA0001C14002000B587B02B49B1F898004FF4AF
:106DB0007A722A490988FCF757FC01284AD12748EA
:106DC00001882548A0F89810D0F8B0000021224A88
:106DD000D2F8B4200B4611431843CDE904101E48E5
:106DE0009030D0E90010DDE90423514058400143C0
:106DF0002FD000210846DDE90432594050400143BC
:106E000027D01748008CADF804009DF8060020F04C
:106E10007F00401D8DF806009DF8060020F08000E0
:106E200080308DF8060001208DF8070000208DF8D5
:106E300008008DF809000B4800680390082204A997
:106E4000684600F0E3FA07480068401C05490860FE
:106E500000BF00BF07B000BD301300202C00002091
:106E60001C140020181400202DE9F04188B00546BC
:106E70000F469046224E00240020079021A103C90E
:106E8000CDE9050121A103C9CDE90301E879401C41
:106E9000E871A87920F08000A87100201D49487190
:106EA00007A808600220C871301901A9FEF771FE19
:106EB0002044C4B210211748417305A815498860C1
:106EC00006211448C173301901A9FEF762FE20445F
:106ED000C4B210210F48417503A80E49086106216C
:106EE0000C48C175301901A9FEF753FE2044C4B205
:106EF000224631462846FFF745FF08B0BDE8F0813D
:106F000008270020504B313134330000303031310C
:106F100038310000CC2C00202DE9F04188B0064625
:106F20000F469046304D0024002007902FA103C942
:106F3000CDE905012FA103C9CDE90301F079401C7A
:106F4000F071B07920F08000B07100208DF8090058
:106F500007A8019002208DF80B00281901A9FEF75F
:106F600018FE2044C4B209208DF8090007A801903A
:106F700001208DF80B00281901A9FEF70AFE204414
:106F8000C4B200208DF8090007A8019002208DF8F6
:106F90000B00281901A9FEF7FCFD2044C4B2102003
:106FA0008DF8090005A8019006208DF80B0028191E
:106FB00001A9FEF7EEFD2044C4B210208DF80900AF
:106FC00003A8019006208DF80B00281901A9FEF7EF
:106FD000E0FD2044C4B2224629463046FFF7D2FEE7
:106FE00008B0BDE8F081000008270020504B313187
:106FF0003433000030303131383100002DE9F04FAA
:1070000089B00746894692469846D54D002007909C
:1070100083460024F879401CF871B87920F080008C
:10702000B8714FF6FF7080457ED100260AE0CD484A
:10703000304100F0010018B10BF1010000F0FF0B2E
:10704000701CC6B2202EF2DB00208DF805000BF17B
:107050000400C0B2079007A800900BF10400C0B272
:107060008DF8070028196946FEF793FD204484B285
:10707000002635E0BB48304100F0010070B300202D
:107080008DF8050007A8009002208DF80700281948
:107090006946FEF77EFD204484B22A208DF8050063
:1070A000039603A8009001208DF80700281969466F
:1070B000FEF76FFD204484B224208DF80500AA4815
:1070C0000690069800EB8600009001208DF80700DE
:1070D00028196946FEF75DFD204484B2701CC6B2D3
:1070E000202EC7DBA048083890F8AC0010B94E201D
:1070F00002900AE09C48083890F8AC00012802D1C0
:107100005320029001E00020029000208DF805003D
:1071100007A8009002208DF8070028196946FEF79D
:1071200038FD204484B200E0E1E02A208DF805001B
:1071300047F23150039003A8009001208DF807001A
:1071400028196946FEF725FD204484B210208DF8E9
:10715000050002A8009001208DF807002819694653
:10716000FEF717FD204484B27F48083890F8AD0040
:1071700010B9522002900AE07B48083890F8AD0020
:10718000012802D15320029001E00020029000204B
:107190008DF8050007A8009002208DF80700281937
:1071A0006946FEF7F6FC204484B22A208DF80500DB
:1071B00047F23250039003A8009001208DF8070099
:1071C00028196946FEF7E5FC204484B210208DF8AA
:1071D000050002A8009001208DF8070028196946D3
:1071E000FEF7D7FC204484B25F48083890F8AE0020
:1071F00010B9522002900AE05B48083890F8AE00BF
:10720000012802D15320029001E0002002900020CA
:107210008DF8050007A8009002208DF807002819B6
:107220006946FEF7B6FC204484B22A208DF805009A
:1072300047F23350039003A8009001208DF8070017
:1072400028196946FEF7A5FC204484B210208DF869
:10725000050002A8009001208DF807002819694652
:10726000FEF797FC204484B23F480838D0F8B000BD
:1072700000213D4A083AD2F8B4200B461143184386
:10728000CDE9041000208DF8050007A80090022029
:107290008DF8070028196946FEF77BFC204484B26C
:1072A0002A208DF8050047F23450039003A800907F
:1072B00001208DF8070028196946FEF76AFC204472
:1072C00084B228208DF8050004A8009001208DF8D4
:1072D000070028196946FEF75CFC204484B2224668
:1072E00029463846FFF74EFD09B0BDE8F08F002073
:1072F0008DF8050007A8009001208DF807002819D7
:107300006946FEF746FC204484B2B8F1010F0DD166
:107310008DF805A0CDF8009001208DF80700281900
:107320006946FEF736FC204484B212E04FF6FF7047
:1073300080450DD18DF805A0CDF8009001208DF885
:10734000070028196946FEF724FC204484B200E0B7
:10735000CAE7224629463846FFF714FD00BFC3E7B7
:1073600008270020FFD97F00381300202DE9FE43B5
:1073700004460F4690460F4E002501200290E0790A
:10738000401CE071A07920F08000A07108200A491B
:10739000487102A808600120C87170196946FEF79B
:1073A000F8FB2844C5B22A4631462046FFF7EAFCDE
:1073B000BDE8FE8308270020CC2C00202DE9FE43E9
:1073C00004460F469046104E002501200290E079B9
:1073D000401CE071A07920F08000A07109208DF898
:1073E000050002A8009001208DF807007019694679
:1073F000FEF7CFFB2844C5B22A4631462046FFF7A8
:10740000C1FCBDE8FE830000082700202DE9F74FEE
:1074100088B089466E4E002400200790824683463D
:107420008DF8090007A8019002208DF80B00301993
:1074300001A9FEF7AEFB204484B2D9E90078CDF86B
:107440001480069700250AE00598E84000F0010046
:1074500018B10AF1010000F0FF0A681C85B2202D66
:10746000F2DB00208DF8090007A801904FEA4A00DE
:10747000401CC0B28DF80B00301901A9FEF789FB42
:10748000204484B208208DF8090005A8019001204D
:107490008DF80B00301901A9FEF77BFB204484B264
:1074A00000252BE00598E84000F0010020B3E8B289
:1074B000049029208DF8090004A8019001208DF87E
:1074C0000B00301901A9FEF764FB204484B21020A0
:1074D0008DF809003F4850F8250001903D4951F8CA
:1074E0002500F8F755FEC0B28DF80B00301901A940
:1074F000FEF74FFB204484B2681C85B2202DD1DBFF
:1075000000250AE00698E84000F0010018B10BF1F0
:10751000010000F0FF0B681C85B2202DF2DB00207B
:107520008DF8090007A801904FEA4B00401CC0B23B
:107530008DF80B00301901A9FEF72BFB204484B213
:1075400008208DF8090006A8019001208DF80B0095
:10755000301901A9FEF71DFB204484B200252DE05F
:107560000698E84000F0010030B305F13200C0B2E7
:10757000039029208DF8090003A8019001208DF8BF
:107580000B00301901A9FEF704FB204484B210203F
:107590008DF80900104850F8250001900E4951F867
:1075A0002500F8F7F5FDC0B28DF80B00301901A9E0
:1075B000FEF7EFFA204484B2681C85B2202DCFDBA1
:1075C000224631460898FFF7DDFB0BB0BDE8F08F8F
:1075D0000827002030120020B012002070B50646A7
:1075E0000C46154629462046FEF77AFB70BD00B9C9
:1075F0007047002141610161C16000BFF8E770B5CB
:1076000004460D460CB9002070BDE06808B90020A2
:10761000FAE745B1D4E90006236903FB06013246C7
:107620002846FEF7A9FA2069401CA16890FBF1F2F8
:1076300001FB12002061E068401EE0600120E3E7EA
:1076400070B504460D460CB9002070BDD4E9021097
:10765000884201D10020F8E745B1D4E900166369FA
:1076600003FB061032462946FEF786FA6069401C85
:10767000A16890FBF1F201FB12006061E068401C20
:10768000E0600120E1E770B504460D460CB900202A
:1076900070BDD4E90210884204DA29462046FFF77B
:1076A000CFFFF5E745B1D4E90016636903FB061087
:1076B00032462946FEF760FA6069401CA16890FBDB
:1076C000F1F201FB120060612069401CA16890FB8F
:1076D000F1F201FB120020610120D9E710B5034649
:1076E00062B9002007E0C0F10104E40043FA04F4A9
:1076F0000C54441CE0B20228F5DB0BE0012A09D14E
:10770000002005E0C40043FA04F40C54441CE0B229
:107710000228F7DB10BD10B5034662B9002007E070
:10772000C0F10304E40023FA04F40C54441CE0B256
:107730000428F5DB0BE0012A09D1002005E0C40094
:1077400023FA04F40C54441CE0B20428F7DB10BD07
:1077500030B50246002361B9002007E0145CC0F197
:107760000105ED00AC402343441CE0B20228F5DBE8
:107770000BE0012909D1002005E0145CC500AC40F4
:107780002343441CE0B20228F7DB98B230BD30B589
:107790000246002361B9002007E0145CC0F1030534
:1077A000ED00AC402343441CE0B20428F5DB0BE0C1
:1077B000012909D1002005E0145CC500AC40234339
:1077C000441CE0B20428F7DB184630BD0203040570
:1077D000060708090A0B0C0D0E0F1010010200001D
:1077E0000000000000000102030406070809000071
:1077F000000001020304DDDDDDDDDCBBBBDDDDDD22
:10780000DDDDDDDDDDDD988888888888888877770C
:107810007777778888888555555666666666666682
:1078200066666668888883333332222222222222C7
:1078300022222228888D000056312E3000000000C0
:10784000456D657267656E6379206F666628454D84
:107850004F290000456D657267656E63792073740A
:107860006F7028454D5329004250206F7665726C29
:107870006F616420320000004D50206F7665726C9D
:107880006F61642032000000436173696E67207489
:10789000656D702E20484800576174657220666CD3
:1078A0006F77206C6F7720636F6E74696E75656497
:1078B000000000005761746572206C65616B616740
:1078C00065000000506F776572206661696C7572A3
:1078D0006500000042502064726976657220707203
:1078E0006F74656374696F6E206163746976650097
:1078F0004D50206472697665722070726F74656392
:1079000074696F6E2061637469766500425020442B
:10791000726F6F70696E67004D502044726F6F70A8
:10792000696E6700436F6F6C657220312074656DFE
:10793000702E206869676800436F6F6C6572203233
:107940002074656D702E206869676800436F6F6CE6
:10795000657220332074656D702E20686967680039
:10796000436173696E672074656D702E2068696766
:10797000680000004472766E206272672074656D44
:10798000702E2068696768004472762062726720F2
:1079900074656D702E206869676800004578682EF0
:1079A00020747261702074656D702E20686967683C
:1079B000000000004472697665722074656D702E57
:1079C00020686967680000004250206D6F746F7214
:1079D0002074656D702E2068696768004D50206DB9
:1079E0006F746F722074656D702E2068696768000F
:1079F0004261636B2070726573732E2068696768DB
:107A000000000000424F582074656D702E68696751
:107A10006800000045787465726E616C20696E7450
:107A200065726C6F636B0000425020746865726D04
:107A3000616C00004D5020746865726D616C0000CF
:107A40004E322076616C7665206F70656E000000A6
:107A500056616C7665206572726F7200436F6D6D52
:107A6000756E69636174696F6E206572726F720002
:107A7000486561746572206572726F720000000063
:107A80004F74686572207761726E696E677300006B
:107A90004F7468657220616C61726D730000000044
:107AA0004250206E6F2063757272656E7400000024
:107AB0004D50206E6F2063757272656E7400000009
:107AC00042502073746570206F7574004D502073A0
:107AD000746570206F7574004F696C206C657665F5
:107AE0006C206C6F7700000042502D47206F696C4E
:107AF000206C6576656C206C6F7700004D502D47CB
:107B0000206F696C206C6576656C206C6F77000067
:107B100042502D4D206F696C206C6576656C206C31
:107B20006F7700004D502D4D206F696C206C65768D
:107B3000656C206C6F7700004578682E204E3220EF
:107B4000666C6F77206C6F770000000050756D7069
:107B5000204E3220666C6F77206C6F77000000003B
:107B600044696C2E4E3220666C6F77206C6F770004
:107B7000576174657220666C6F77206C6F770000B8
:107B800000000000A47B0008000000206C1400002E
:107B9000840E0008A47D00086C140020042400005A
:107BA0000C470008413210420113127A133878183A
:107BB000120853454353322056312E302D56302E65
:107BC000303009011D1008C0A80101FFFFFF150C8E
:107BD00029AB7C1A010E0A13651503FF138801FFF8
:107BE00001FF01FF01FF01FF01FF01FF01FF01FF95
:107BF00001FF01FF01FF01FF01FF01FF012713E169
:107C0000571B089504130D5A1408B1432308441454
:107C100020F1551B08D1041390164320013905A10A
:107C20000B159017185A1818E20213A0101420D040
:107C3000141420A4151B206004293913901C1C2047
:107C4000901D0C4A014632141357561B08438C1AD8
:107C50008F041A770C1A1D08411ABD0C1AB844E19A
:107C600019441A1E440A281F441AD0441A18801AAC
:107C70002CD86AE8881A20441A240C4A04B6091E33
:107C80004413115B1B0801048BB4119013E14B14D6
:107C900008754C1408394D9B08C01801241335543D
:107CA0001C089D534019048113902633200CF20ABE
:107CB00013707B1B0880041A6004130C791B0818CE
:107CC000041A600413E87A1B0810141AFC081A241A
:107CD000081A88141A74041AD8101A04042A4018AE
:107CE00019101A38042A4C0419241A38041A9C0C46
:107CF0001AF0041A70201AC8081ADC041AB4041AFC
:107D00005C101A5004296C790419109B8878281982
:107D10000C1A2814DA34281A54181AB0145AA01855
:107D200029601AC4141AF0041AD4041A68041A78C0
:107D3000041AC0202ACC9C190C298C1A9808EA1421
:107D40007499041A901C1318120397200713B95E34
:107D50008208D4FFD97F13655F1B0885041AFD24B0
:107D60001A19081A39041AA5041AC90413556614F5
:107D70000830131C20B96914126D14080C14022861
:107D80002013D15C1B0831541A1C34320113F13119
:107D90001C086D354819141AB50413A5325B084C3C
:047DA000500000008F
:04000005080000ED02
:00000001FF
